:020000040800F2
:1000000060080020D5010008C1660008C36600082A
:10001000C7660008CB660008CF6600080000000035
:10002000000000000000000000000000D36600088F
:10003000D566000800000000D7660008ED01000842
:10004000EF010008EF010008EF010008EF010008D0
:10005000EF010008EF010008EF010008EF010008C0
:10006000EF010008EF010008EF010008EF010008B0
:10007000EF010008EF010008EF010008EF010008A0
:10008000EF010008EF010008EF010008EF01000890
:10009000EF010008EF010008EF010008EF01000880
:1000A000EF010008EF010008EF010008EF01000870
:1000B00009260008EF010008F1250008EF010008FB
:1000C000EF010008EF010008EF010008EF01000850
:1000D000EF010008CD1F0008512C0008EF010008B7
:1000E000EF010008EF010008EF010008EF01000830
:1000F000EF010008EF010008EF010008EF01000820
:10010000EF010008EF010008EF010008EF0100080F
:10011000EF010008EF010008D3260008EF010008F6
:10012000EF010008EF010008EF010008EF010008EF
:1001300000F002F800F03FF80AA090E8000C8244BA
:100140008344AAF10107DA4501D100F034F8AFF297
:10015000090EBAE80F0013F0010F18BFFB1A43F0A5
:1001600001031847848C0000A48C0000103A24BFBF
:1001700078C878C1FAD8520724BF30C830C144BF0C
:1001800004680C607047000000230024002500264E
:10019000103A28BF78C1FBD8520728BF30C148BFEA
:1001A0000B607047642906F0FD82002070471FB580
:1001B0001FBD10B510BD06F0B5FC1146FFF7F7FFE7
:1001C00006F0B8F906F0D3FC03B4FFF7F2FF03BC66
:1001D00001F0B4FE0948804709480047FEE7FEE702
:1001E000FEE7FEE7FEE7FEE7FEE7FEE7FEE7FEE7E7
:1001F00004480549054A064B70470000F302000811
:100200003101000860020020600800206004002026
:10021000600400200CB50020019000906C4800683C
:1002200040F480306A49086000BF6948006800F403
:10023000003000900198401C0190009818B9019876
:10024000B0F5A06FF1D16248006800F4003010B141
:100250000120009001E0002000900098012843D187
:100260005C48006840F010005A4908600846006881
:1002700020F0030008600846006840F002000860B3
:1002800053484068524948600846406848600846FC
:10029000406840F4806048600846406820F47C1064
:1002A00048600846406840F4E81048600846006826
:1002B00040F08070086000BF4548006800F00070A2
:1002C0000028F9D04248406820F0030040494860C7
:1002D0000846406840F00200486000BF3C48406863
:1002E00000F00C000828F9D10CBD10B5FFF792FF03
:1002F00010BD10B53648006840F001003449086070
:10030000084640683449084031494860084600685A
:10031000324908402E4908600846006820F48020D1
:1003200008600846406820F4FE0048604FF41F0053
:100330008860FFF7DAFF4FF000602949086010BDC0
:1003400010B5002100200022214B5B6803F00C0156
:1003500021B1042906D0082928D107E0214B224CDD
:10036000236027E01F4B204C236023E0184B5B6881
:1003700003F47010164B5B6803F48032022303EB26
:10038000904022B9194B4343174C23600DE0104BAA
:100390005B6803F4003323B1144B4343124C2360D6
:1003A00003E0104B4343104C236003E00D4B0E4C15
:1003B000236000BF00BF064B5B68C3F303130C4C04
:1003C000E15C094B1B68CB40074C236010BD00006B
:1003D00000100240002002400000FFF8FFFFF6FE80
:1003E00008ED00E000127A000000002000093D0046
:1003F0000400002031490143314A1160704770B553
:10040000002100230F22C47804B32D4C246804F487
:10041000E064C4F5E064210AC1F10403CA404478F1
:1004200004FA03F18478144021430901254C06782D
:10043000A155047804F01F050124AC4005786D1126
:10044000AD0005F1E025C5F8004109E0047804F0AD
:100450001F050124AC401C4D0678761145F8264056
:1004600070BD1A4A0A400243154B1B1F1A607047A1
:1004700039B1134A121D12680243114B1B1D1A6039
:1004800006E00F4A121D126882430D4B1B1D1A60B5
:100490007047042808D14FF0E021096941F00401B8
:1004A0004FF0E022116107E04FF0E021096921F0EF
:1004B00004014FF0E0221161704700000000FA05CE
:1004C0000CED00E000E400E080E100E080FFFF1FB1
:1004D00010B50446CC48844208D10121042000F024
:1004E0002DFB0021042000F029FB46E0C748844290
:1004F00008D10121082000F021FB0021082000F094
:100500001DFB3AE0C248844208D10121102000F0CE
:1005100015FB0021102000F011FB2EE0BD488442A5
:1005200008D10121202000F009FB0021202000F04B
:1005300005FB22E0B848844208D10121402000F0A8
:10054000FDFA0021402000F0F9FA16E0B348844299
:1005500008D10121802000F0F1FA0021802000F074
:10056000EDFA0AE0AE48844207D10121801500F07F
:10057000E5FA0021A01500F0E1FA10BD10B5012147
:10058000084600F0DBFA0021012000F0D7FA10BD88
:100590002DE9F0410246002500260020002300241A
:1005A000002791F803C00CF00F0591F803C00CF080
:1005B000100CBCF1000F03D091F802C04CEA050505
:1005C00091F800C0BCF1000F31D0146800202BE07E
:1005D0004FF0010C0CFA00F3B1F800C00CEA03066E
:1005E0009E4220D183004FF00F0C0CFA03F7BC435E
:1005F00005FA03FC4CEA040491F803C0BCF1280F8F
:1006000006D14FF0010C0CFA00FCC2F814C00AE04D
:1006100091F803C0BCF1480F05D14FF0010C0CFA62
:1006200000FCC2F810C0401C0828D1D31460B1F8F7
:1006300000C0BCF1FF0F34DD546800202EE000F153
:10064000080C4FF0010808FA0CF3B1F800C00CEAEE
:1006500003069E4221D183004FF00F0C0CFA03F7E2
:10066000BC4305FA03FC4CEA040491F803C0BCF156
:10067000280F05D100F1080C08FA0CF8C2F8148014
:1006800091F803C0BCF1480F07D100F1080C4FF0FE
:10069000010808FA0CF8C2F81080401C0828CED3D4
:1006A0005460BDE8F0814FF6FF7101800221817036
:1006B0000421C17070470246002093680B400BB1C3
:1006C000012000E0002070470146886880B2704732
:1006D00002460020D3680B400BB1012000E000204F
:1006E00070470146C86880B2704701617047416138
:1006F00070470AB1016100E041617047C160704715
:100700004FF480320A438261816182618269826929
:10071000704702460020434B18684FF6807318401C
:1007200040EA021008433F4B186070473E49C861D9
:100730007047F0B50A46002300240021002500F090
:100740000046B6F1004F02D1364EF16901E0354E58
:100750007168C0F3034583B200F44016B6F5401F3C
:1007600008D121F070612F4E766826F070662D4F0B
:100770007E6012E000F48016B6F5801F06D10326D5
:1007800006FA05F4A14341F0706106E0460D36011A
:1007900003FA06F6B14341F0706122B1460D36010D
:1007A00003FA06F6314300F00046B6F1004F02D1DD
:1007B0001C4EF16101E01B4E7160F0BD30B50022AE
:1007C0008B071C0F0F2303FA04F2164B08338C100F
:1007D00053F824309343134C08348D1044F82530DB
:1007E00023468C1053F824308C07240F00FA04F4AD
:1007F00023430C4C08348D1044F8253030BD0A4991
:10080000DC3108607047000000080140000C014026
:10081000001001400014014000180140001C01407C
:10082000002001400000014000002042DF48006835
:1008300040F00100DD49086008464068DC49084096
:10084000DA49486008460068DA490840D749086034
:100850000846006820F4802008600846406820F4BC
:10086000FE0048604FF41F0088607047CF49096858
:1008700021F48031CD4A11601146096821F48021AC
:100880001160B0F5803F03D0B0F5802F0ED106E0A7
:10089000C649096841F48031C44A116007E0C34980
:1008A000096841F4A021C14A116000E000BF00BF07
:1008B000704710B501460022002300204A11012A8A
:1008C00002D1BA4C236806E0022A02D1B74C236A4F
:1008D00001E0B64C636A01F01F02012494401C4001
:1008E0000CB1012000E0002010BD38B500200090C0
:1008F0000024002500BF3120FFF7DBFF05460098EC
:10090000401C00900098B0F5A06F01D0002DF2D0EF
:100910003120FFF7CEFF08B1012400E0002420467B
:1009200038BD01460020A14A106820F0F80040EAD6
:10093000C10010607047A04908607047024600205F
:100940009A4B586820F47C1042EA01031843974BF5
:100950005860704798490866704701460020934ADE
:10096000506820F003000843506070478F4840688B
:1009700000F00C007047014600208C4A506820F0BF
:10098000F00008435060704701460020874A5068D5
:1009900020F4E06008435060704701460020834A1D
:1009A000506820F4605040EAC1005060704729B19F
:1009B0007E4A527A02437D4B5A7204E07B4A527A55
:1009C00082437A4B5A7270477B49D831086070472E
:1009D00001460020754A506820F4404008435060AA
:1009E00070470021714A20321170704A82F820103D
:1009F000012802D004280AD104E001216B4A2032E8
:100A0000117005E00521694A2032117000E000BF35
:100A100000BF70476949086070476449096A01432B
:100A2000624A11627047654944390860704730B5C1
:100A300000210022002400235C4D6D6805F00C01AC
:100A400021B1042905D0082923D105E05C4D0560BA
:100A500022E05B4D05601FE0544D6D6805F4701297
:100A6000524D6D6805F48034022505EB92421CB9A5
:100A7000544D554305600BE04C4D6D6805F4003551
:100A80001DB1504D5543056002E04D4D5543056085
:100A900002E04B4D056000BF00BF444D6D6805F09E
:100AA000F0010909484D6B5C0568DD4045603F4D2C
:100AB0006D6805F4E061090A434D6B5C4568DD40F3
:100AC00085603A4D6D6805F46051C90A3E4D6B5C16
:100AD0004568DD40C560354D6D6805F44041890BC2
:100AE0003A4D6B5CC568B5FBF3F5056130BD29B1C6
:100AF0002E4A526902432D4B5A6104E02B4A526937
:100B000082432A4B5A61704729B1284A92690243AD
:100B1000264B9A6104E0254A92698243234B9A61ED
:100B2000704729B1214AD2690243204BDA6104E0BF
:100B30001E4AD26982431D4BDA61704729B11B4AB4
:100B4000D2680243194BDA6004E0184AD268824343
:100B5000164BDA60704729B1144A12690243134BED
:100B60001A6104E0114A12698243104B1A617047FE
:100B700012494039086070470F49C86470470B49F3
:100B8000C87170470948406A40F080700749486260
:100B9000704701460020054A92680A400AB10120C8
:100BA00000E0002070470149887270470010024041
:100BB0000000FFF8FFFFF6FE0000424280044242C0
:100BC00000127A0000093D001400002024000020DB
:100BD00010B50446FE48844208D10121C014FFF735
:100BE000ADFF0021E014FFF7A9FFC4E0B4F1804F8E
:100BF00008D101210846FFF7AEFF00210120FFF7D1
:100C0000AAFFB8E0F348844208D101210220FFF78F
:100C1000A2FF00210220FFF79EFFACE0EE488442D5
:100C200008D101210420FFF796FF00210420FFF7DF
:100C300092FFA0E0E948844208D101210820FFF793
:100C40008AFF00210820FFF786FF94E0E4488442F1
:100C500008D101211020FFF77EFF00211020FFF7AF
:100C60007AFF88E0DF48844208D101212020FFF785
:100C700072FF00212020FFF76EFF7CE0DA488442FB
:100C800008D101214014FFF759FF00216014FFF73C
:100C900055FF70E0D548844209D10121C804FFF70F
:100CA0004DFF00214FF40020FFF748FF63E0D048DC
:100CB000844209D101210805FFF740FF00214FF4CC
:100CC0008010FFF73BFF56E0CA48844209D101215A
:100CD0004805FFF733FF00214FF40010FFF72EFF08
:100CE00049E0C548844208D101214020FFF733FF85
:100CF00000214020FFF72FFF3DE0C048844208D18B
:100D000001218020FFF727FF00218020FFF723FF2C
:100D100031E0BB48844208D101218015FFF71BFF59
:100D20000021A015FFF717FF25E0B648844209D13E
:100D300001210804FFF702FF00214FF48030FFF784
:100D4000FDFE18E0B048844209D101214804FFF7B4
:100D5000F5FE00214FF40030FFF7F0FE0BE0AB484A
:100D6000844208D101218804FFF7E8FE00214FF4F6
:100D70008020FFF7E3FE10BD00220288944B9842CA
:100D80000ED0994B98420BD0B0F1804F08D0914BC8
:100D9000984205D0904B984202D0904B984204D193
:100DA0004FF68F731A404B881A438D4B984207D0E9
:100DB0008C4B984204D04FF6FF431A40CB881A431D
:100DC00002808B8883850B880385814B98420BD0EA
:100DD000854B984208D08B4B984205D08A4B98425D
:100DE00002D08A4B984201D10B7A03860123838279
:100DF000704770B5002400220023058C4FF6FE7664
:100E000035400584028C8388048B4FF68F752C4007
:100E1000B51E2C400D882C43751E2A400D892A438F
:100E20004D882A436A4DA8420BD06F4DA84208D086
:100E3000744DA84205D0744DA84202D0734DA8420B
:100E400013D14FF6F7752A404D892A434FF6FB75AB
:100E50002A408D882A434FF6FF652B404FF6FF55F9
:100E60002B408D892B43CD892B4383800483CD88F0
:100E70008586028470BD70B5002400220023058C95
:100E80004FF6EF7635400584028C8388048B48F654
:100E9000FF752C404FF6FF452C400D884FF6FF762E
:100EA00006EA05252C434FF6DF752A400D8906EA30
:100EB00005152A434D8806EA05152A43444DA842E4
:100EC00002D0494DA8421DD14FF67F752A404D8969
:100ED0004FF6FF7606EA05152A434FF6BF752A40FE
:100EE0008D8806EA05152A434FF6FF352B404FF251
:100EF000FF752B408D8906EA85052B43CD8906EACF
:100F000085052B4383800483CD880587028470BDCB
:100F100070B5002400220023058C4FF6FF66354093
:100F20000584028C8388848B4FF68F752C404FF696
:100F3000FC752C400D882C434FF6FF552A400D8937
:100F40004FF6FF7606EA05252A434D8806EA052571
:100F50002A431F4DA84202D0234DA8421DD14FF273
:100F6000FF752A404D894FF6FF7606EA05252A438C
:100F70004FF6FF352A408D8806EA05252A434EF6AE
:100F8000FF752B404DF6FF752B408D8906EA051540
:100F90002B43CD8906EA05152B4383808483CD88B6
:100FA0008587028470BD70B5002200230024058C63
:100FB0004EF6FF7635400584038C8488828B48F694
:100FC000FF752A404FF6FF452A400D8820E00000BB
:100FD000002C01400004004000080040000C0040CC
:100FE000001000400014004000340140004C01405B
:100FF000005001400054014000180040001C004017
:1010000000200040004001400044014000480140F1
:101010004FF6FF7606EA05252A434DF6FF752B406D
:101020000D8906EA05352B434D8806EA05352B4325
:10103000FA4DA84202D0FA4DA84208D14BF6FF75EE
:101040002C408D894FF6FF7606EA85152C43848067
:101050008283CD88A0F84050038470BD828B4FF20C
:10106000FF331A408283828B4FF6FF7303EA01231A
:101070001A4382837047F0B50C46154600220021C2
:101080000026078C4EF6FF7C07EA0C070784828B4C
:10109000018C4FF6FF7707EA043640F6FF473A40E7
:1010A0004FF6FF7707EA05273A434FF6FF7707EA3F
:1010B00003373A43D94FB8420ED0D94FB8420BD07C
:1010C000B0F1804F08D0D74FB84205D0D64FB842C4
:1010D00002D0D64FB84206D14DF6FF77394046F4DC
:1010E0008057394305E047F6FF57394044F48057AD
:1010F000394382830184F0BD828B4FF6F3731A402B
:101100008283828B0A4382837047F0B50C46154672
:10111000002200210026078C4FF6FF6C07EA0C071F
:101120000784828B018C4FF6FF7707EA04264FF67F
:101130000C773A404FF6FF7707EA03172F433A43FD
:10114000B64FB8420ED0B64FB8420BD0B0F1804F78
:1011500008D0B44FB84205D0B34FB84202D0B34F15
:10116000B84206D14FF6FF57394046F480773943ED
:1011700005E04FF2FF57394044F4807739438283CA
:101180000184F0BD028B4FF2FF331A400283028BC1
:101190004FF6FF7303EA01231A4302837047F0B549
:1011A0000C461546002200210026078C4FF6EF7CE6
:1011B00007EA0C070784028B018C4FF6FF7707EADA
:1011C000041640F6FF473A404FF6FF7707EA033729
:1011D0003A434FF6FF7707EA05273A438F4FB84265
:1011E0000ED08F4FB8420BD0B0F1804F08D08D4F4A
:1011F000B84205D08C4FB84202D08C4FB84206D1CD
:101200004FF6DF77394046F01007394305E04FF6D7
:101210005F77394044F01007394302830184F0BD01
:10122000028B4FF6F3731A400283028B0A43028348
:101230007047F0B50C46154600220021068C4FF68B
:10124000FE773E400684028B018C4FF60C763240CE
:101250007E1C06EA03162E433243704EB0420ED077
:101260006F4EB0420BD0B0F1804F08D06D4EB042FF
:1012700005D06D4EB04202D06C4EB04206D14FF652
:10128000FD76314044F00106314305E04FF6F57636
:10129000314044F00106314302830184F0BD70B552
:1012A00005460C465D4885420ED05D4885420BD010
:1012B000B5F1804F08D05B48854205D05A48854239
:1012C00002D05A48854200D100E000BF208850B9C2
:1012D0002389A28861882846FFF7ABFFE18828466A
:1012E000FFF79EFF25E0208804280AD12389A288E1
:1012F00061882846FFF753FFE1882846FFF742FF41
:1013000017E0208808280AD12389A2886188284606
:10131000FFF7FBFEE1882846FFF7EEFE09E0238990
:10132000A28861882846FFF7A6FEE1882846FFF7D5
:1013300095FE70BD2DE9F04105460C4600260127BB
:10134000608808B9022600E00026A088012801D1A3
:10135000022700E001272088A0B92389A28861889C
:101360002846FFF766FFE1882846FFF759FF2389E3
:101370003A4631462846FFF712FFE1882846FFF734
:1013800001FF13E02389A28861882846FFF707FF41
:10139000E1882846FFF7F6FE23893A46314628467B
:1013A000FFF747FFE1882846FFF73AFFBDE8F081E5
:1013B0000A884B881A438B881A43CB881A430B89B7
:1013C0001A434B891A438B891A43A0F8442070476B
:1013D0004FF6FF71818000210180C1804180017240
:1013E00070470021018041808180C180018141815D
:1013F0008181C1817047002101804180012181806C
:101400000021C180018170470021018041808180DD
:10141000C18001814181818170470000002C014021
:10142000003401400004004000080040000C00406F
:1014300021B1028842F00102028004E002884FF6E6
:10144000FE731A400280704731B1B0F8442042F474
:101450000042A0F8442005E0B0F84420C2F30E0298
:10146000A0F8442070471AB183890B43838102E0BE
:1014700083898B43838170478182704741EA0203ED
:10148000A0F8483070471AB183890B43838102E08A
:1014900083898B438381704701894FF6F87211402D
:1014A000018170470A46002101894FF68F73194068
:1014B00011430181704730B504460D462946204648
:1014C000FFF7F0FF208940F00700208130BD2DE9B3
:1014D000F04104460D4616461F46602D06D13B4698
:1014E000012231462046FFF75AFE05E03B46012225
:1014F00031462046FFF79DFE29462046FFF7D2FFE2
:10150000208940F007002081BDE8F08130B50C460D
:1015100000210189C9B24FF6FF7505EA032515437D
:1015200025432943018130BD2DE9F04105460E4692
:1015300017469846002443463A4631462846FFF768
:10154000E5FF2C894FF6F870044044F007044FF68D
:101550008F70044044F070042C81BDE8F081F0B538
:1015600004460D4616461F463B463246294620464F
:10157000FFF7CCFF208940F480402081F0BD018539
:10158000828270470A46002101884FF68F73194006
:10159000114301807047F0B50C4615461E460021E8
:1015A000002200230189028B038C4FF6F877394023
:1015B00021434FF6FC473A4040F201173A434FF6B9
:1015C000DD773B404FF6FF7707EA06172F433B4393
:1015D000018102830384F0BD0A460021018B4FF68E
:1015E0008F7319401143018370470A460021018B14
:1015F00048F6FF7319404FF6FF7303EA02231943BD
:10160000018370470A460021818B4FF68F73194082
:101610001143818370470A460021818B48F6FF738E
:1016200019404FF6FF7303EA022319438183704781
:1016300021B1028842F08002028004E002884FF665
:101640007F731A400280704721B1828842F0040201
:10165000828004E082884FF6FB731A4082807047D4
:1016600021B1828842F00802828004E082884FF62D
:10167000F7731A408280704721B1828842F00102DC
:10168000828004E082884FF6FE731A4082807047A1
:101690000A460021018B4FF6F7731940114301836D
:1016A00070470A460021018B4FF2FF7319404FF635
:1016B000FF7303EA02231943018370470A4600219E
:1016C000818B4FF6F77319401143818370470A46A7
:1016D0000021818B4FF2FF7319404FF6FF7303EA2D
:1016E00002231943818370470A460021018B4FF67C
:1016F000FB7319401143018370470A460021018B97
:101700004FF6FF3319404FF6FF7303EA02231943E4
:10171000018370470A460021818B4FF6FB73194005
:101720001143818370470A460021818B4FF6FF33B6
:1017300019404FF6FF7303EA022319438183704770
:101740000A460021018B4FF67F7319401143018334
:1017500070470A460021018BC1F30E014FF6FF735B
:1017600003EA02231943018370470A460021818B53
:101770004FF67F7319401143818370470A46002159
:10178000818BC1F30E014FF6FF7303EA0223194365
:10179000818370470A460021018C4FF6FD73194082
:1017A0001143018470470A460021018C4FF6F773FC
:1017B00019401143018470470A460021018C4FF6FD
:1017C000DF7319404FF6FF7303EA021319430184D4
:1017D00070470A460021018C4FF67F7319404FF67F
:1017E000FF7303EA02131943018470470A4600217C
:1017F000018C4FF6FF5319404FF6FF7303EA0223A3
:101800001943018470470A460021018C4FF2FF738F
:1018100019404FF6FF7303EA02231943018470470E
:101820000A460021018C4DF6FF7319404FF6FF73F5
:1018300003EA023319430184704730B500230124C1
:101840008C40A3B2048C9C430484048C02FA01F5FE
:10185000ADB22C43048430BD30B5002304248C4049
:10186000A3B2048C9C430484048C02FA01F5ADB24B
:101870002C43048430BD70B5034600200024184674
:10188000183001258D40ACB21D8CA5431D8409B1D3
:10189000082909D100EB6100056825F07005056095
:1018A0000568154305600EE00D1FC5F34E0528447D
:1018B000056825F4E045056005684FF6FF7606EA01
:1018C00002263543056070BD21B1028842F0020254
:1018D000028004E002884FF6FD731A4002807047D0
:1018E00021B1028842F00402028004E002884FF62F
:1018F000FB731A400280704721B1828842F0800257
:10190000828004E082884FF67F731A40828070479D
:1019100002884FF6F7731A40028002880A43028059
:10192000704782884FF68F731A40828082880A43FC
:101930008280704702894FF6F8731A40028102894B
:101940000A430281704702894FF67F731A40028171
:1019500002890A43028170478184704781857047FC
:10196000818670470187704781877047A0F84010D3
:10197000704702884FF6FF431A40028002880A43EC
:10198000028070470146888E70470146088F704775
:101990000146888F70470146B1F840007047014604
:1019A000888C70470146088D704702460020138AD4
:1019B0000B400BB1012000E000207047CA430282B7
:1019C000704730B50246002000230024158A05EA3E
:1019D0000103958905EA010413B10CB1012000E06F
:1019E000002030BDCA4302827047000010B5044693
:1019F000FB48844209D101218803FFF79FF80021A9
:101A00004FF48040FFF79AF832E0F648844209D15B
:101A100001214804FFF79FF800214FF40030FFF741
:101A20009AF825E0F048844209D101218804FFF7A3
:101A300092F800214FF48020FFF78DF818E0EB4872
:101A4000844209D10121C804FFF785F800214FF431
:101A50000020FFF780F80BE0E548844208D101211F
:101A60000805FFF778F800214FF48010FFF773F8AE
:101A700010BD2DE9F04786B005460E460024A2466B
:101A800000BFA1460027B08900B100BF2F462C8AB5
:101A90004CF6FF700440F08804432C82AC894EF66B
:101AA000F3100440B0883189084371890843044326
:101AB000AC81AC8A4FF6FF400440B0890443AC824D
:101AC00001A8FEF7B4FFC648874202D1DDF810A096
:101AD00001E0DDF80CA0A88900F4004040B10AEB59
:101AE000CA0000EB0A1031684900B0FBF1F807E0CA
:101AF0000AEBCA0000EB0A1031688900B0FBF1F86C
:101B00006420B8FBF0F004012009642101FB108976
:101B1000A88900F4004040B1322000EBC900B0FBBE
:101B2000F1F000F00700044308E0322000EB091058
:101B30006421B0FBF1F000F00F0004432C8106B0EB
:101B4000BDE8F0874FF41651016000218180C1800B
:101B500001810C21418100218181704710B502462D
:101B60000020108A4FF2FF0318400B884C88234353
:101B70008C882343CC8823431843108210BD002156
:101B8000018041808180C180704721B1828942F407
:101B90000052828104E082894DF6FF731A408281EF
:101BA0007047F0B50346002400260025002040F6CB
:101BB0006A17B94200D100BF1846C1F3421401F0C0
:101BC0001F06012707FA06F5012C01D10C3004E0AD
:101BD000022C01D1103000E014301AB107682F43F5
:101BE000076002E00768AF430760F0BD1AB1838A5F
:101BF0000B43838202E0838A8B4383827047028A8D
:101C00004FF6F0731A400282028A0A43028270473A
:101C100082894FF2FF731A40828182890A4382814E
:101C2000704721B1828942F00202828104E08289F8
:101C30004FF6FD731A4082817047028A4FF6DF73B8
:101C40001A400282028A0A430282704721B1028A44
:101C500042F48042028204E0028A4BF6FF731A408B
:101C600002827047C1F3080282807047014688886B
:101C7000C0F308007047818941F0010181817047FC
:101C8000028BD2B20283028B42EA012202837047A6
:101C9000028B02F47F420283028B0A430283704765
:101CA00021B1828A42F02002828204E0828A4FF6C9
:101CB000DF731A408282704721B1828A42F010029B
:101CC000828204E0828A4FF6EF731A408282704764
:101CD00021B1828A42F00802828204E0828A4FF6B1
:101CE000F7731A408282704721B1828942F4004220
:101CF000828103E08289C2F30E028281704721B1A2
:101D0000828A42F40062828204E0828A4FF2FF7388
:101D10001A4082827047828A4FF6FB731A40828291
:101D2000828A0A438282704721B1828A42F002028B
:101D3000828204E0828A4FF6FD731A4082827047E5
:101D400002460020B1F5007F00D100BF13880B4090
:101D50000BB1012000E00020704701F40072B2F5E1
:101D6000007F00D100BFCA430280704770B50246B1
:101D7000002400230025002040F66A16B14200D15D
:101D800000BFC1F3421501F01F03012606FA03F359
:101D9000012D02D19689334006E0022D02D1168A28
:101DA000334001E0968A33400C12012606FA04F40F
:101DB0001688344013B10CB1012000E0002070BD42
:101DC00010B50022002340F66A14A14200D100BFE2
:101DD0000A1201249440A3B2DC43048010BD000029
:101DE000003801400044004000480040004C0040E2
:101DF0000050004070B5482000F016F900F05EF881
:101E000000F028F84FF4E13000F05AF800F04EFFEF
:101E1000002140F60F6000F069FA00F024FB47F261
:101E200030504FF08041888400F06CFB47F2305016
:101E3000064908806421084600F0BAFA4FF4FA75A2
:101E40002C4603480580001D048070BD2408004016
:101E50003C04004008B501211020FEF755FE4FF468
:101E60008070ADF8000010208DF8030003208DF87D
:101E7000020069460F48FEF78BFB08BD70B50446AB
:101E80000D480068401C0C490860A04210D14FF476
:101E900080710848FEF70FFCC0F10100C5B22A4668
:101EA0004FF480710348FEF724FC002002490860CB
:101EB00070BD0000001001402800002070470000A5
:101EC00010B586B00446012144F20400FEF71CFE62
:101ED0004FF40070ADF8140018208DF8170003209F
:101EE0008DF8160005A94B48FEF752FB4FF48060B1
:101EF000ADF8140004208DF8170005A94548FEF739
:101F000047FB01940020ADF80800ADF80A00ADF8D9
:101F10000C00ADF810000C20ADF80E0001A93E48F1
:101F2000FFF7A7FD012240F225513B48FFF739FE9C
:101F300001213948FFF729FE06B010BD00BF7047E8
:101F400000BF354A128802F04002002AF9D0C2B21E
:101F5000314B1B1D1A80704710B5044600BF20216D
:101F60002D48FFF7EDFE0028F9D02B48FFF77EFE45
:101F700010BD70B504460D4640212748FFF7EDFE21
:101F800080212548FFF71CFF13E021782248FFF746
:101F900069FE00BF40212048FFF7D2FE0128F9D199
:101FA00040211D48FFF7D9FE80211B48FFF708FF9D
:101FB000641C281EA5F10105E7D170BD0022174B56
:101FC0001A60174A1160174A1060704710B540F246
:101FD00025511148FFF7CAFED8B10F48FFF746FE5A
:101FE000C4B20F4800680D49096888420CD90D48F1
:101FF000006804700B480068401C0A4908600748E4
:102000000068401C0549086040F225510248FFF76E
:10201000D7FE10BD0008014000380140300000200C
:10202000340000202C00002010B504466FF004009E
:10203000FEF72FFAE11704EB5171C1F3C701234AF0
:1020400011701046007800EB4001C1EBC0104FF654
:10205000FF7101EAC0001E49088010BD01461C4AFC
:1020600012884A434FF0E0235A6100229A6101220C
:102070001A6100BF4FF0E022106900F001021AB1AE
:1020800000F48032002AF5D000224FF0E0231A61DC
:102090009A61704701460D4A12784A434FF0E02397
:1020A0005A6100229A6101221A6100BF4FF0E022BA
:1020B000106900F001021AB100F48032002AF5D054
:1020C00000224FF0E0231A619A6170473C00002023
:1020D0003E000020002001E0411CC8B20A28FBDBC2
:1020E000704710B54FF400617F48FEF7FEFA4FF4D9
:1020F00080617D48FEF7F9FAFFF7ECFF4FF40061CD
:102100007948FEF7F4FAFFF7E5FF4FF4806176486F
:10211000FEF7EDFAFFF7DEFF10BD10B54FF40061DA
:102120007148FEF7E4FA4FF480616F48FEF7DDFA7C
:10213000FFF7D0FF4FF400616B48FEF7D6FA10BDF1
:1021400070B50446002528E004F0800028B14FF463
:1021500000616548FEF7C9FA04E04FF40061624887
:10216000FEF7C5FAFFF7B6FF4FF480615E48FEF751
:10217000BCFAFFF7AFFF4FF480615B48FEF7B7FA98
:10218000072D04D14FF400615748FEF7AEFA600600
:10219000040EFFF79FFF681CC5B2082DD4DB70BD8D
:1021A00010B54FF400615048FEF7A1FAFFF792FF17
:1021B0004FF480614C48FEF798FAFFF78BFF4FF41D
:1021C00080614948FEF793FAFFF784FF4FF40061FE
:1021D0004548FEF78AFA10BD10B54FF40061424839
:1021E000FEF783FAFFF776FF4FF480613E48FEF773
:1021F0007CFAFFF76FFF4FF480613B48FEF777FAF8
:10220000FFF768FF10BD70B505460024002619E0F1
:102210006006040E4FF480613348FEF766FAFFF75C
:1022200059FF4FF400613048FEF745FA08B1601CD1
:10223000C4B24FF480612C48FEF759FAFFF74AFF09
:10224000701CC6B2082EE3DB15B9FFF7C5FF01E02D
:10225000FFF7A6FF204670BD10B54FF4006122487D
:10226000FEF743FAFFF736FF4FF480611E48FEF792
:102270003CFAFFF72FFF4FF400611B48FEF71BFAF3
:1022800008B1012400E000244FF480611648FEF7F5
:102290002EFAFFF71FFF204610BD08B501210820C8
:1022A000FEF732FC4FF44060ADF8000003208DF8DB
:1022B000020014208DF8030069460B48FEF768F908
:1022C000FFF72BFF08BD70B50446FFF7E6FFFFF7E9
:1022D00008FF2046FFF734FFFFF7BEFF0546FFF774
:1022E0001CFF284670BD0000000C014030B589B0CD
:1022F00005460C4601210220FEF713FC681E80B241
:10230000ADF80800A0B2ADF804000020ADF80A0056
:10231000ADF8060001A9C248FEF72EFD0121C04814
:10232000FFF74CFB01221146BD48FFF79CF8012145
:102330000820FEF7E9FB0320ADF8100018208DF807
:10234000130003208DF8120004A9B648FEF720F907
:102350006020ADF814000120ADF816000020ADF8A3
:102360001A00ADF81C0005A9AD48FEF7D1FD082103
:10237000AB48FFF73BFA6020ADF814000120ADF840
:1023800016000020ADF81A00ADF81C0005A9A448FD
:10239000FEF709FE0821A248FFF742FA0121A048F2
:1023A000FFF746F901219E48FFF742F809B030BD1A
:1023B0007FB505460C466020ADF800000120ADF861
:1023C0000200ADF8065069469548FEF7A1FD0821C8
:1023D0009348FFF70BFAADF8064069469048FEF7C0
:1023E000E2FD08218E48FFF71BFA01218C48FFF718
:1023F0001FF97FBD1FB501211020FEF792FB42F2AD
:102400000F70ADF8080040F2CF20ADF804000020B6
:10241000ADF80A00ADF806008DF80C0001A982485D
:10242000FEF7AAFC01218048FFF7C8FA01221146F5
:102430007D48FFF718F84FF44070FDF7DBFF3620BA
:102440008DF8000005208DF8010000208DF80200B5
:1024500001208DF803006846FDF7D1FF0121724885
:10246000FEF7E6FF1FBD00B587B001210846FEF765
:1024700058FB01210420FEF747FB0320ADF80000C4
:1024800004208DF8030069466848FEF781F804A827
:10249000FEF79EFF0020ADF810004EF66020ADF86C
:1024A00014004FF40070ADF816000020ADF81200D3
:1024B00004A94FF08040FEF75FFC00231A46032179
:1024C0004FF08040FFF767F801A8FEF794FF0A205D
:1024D000ADF80C0001A94007FEF7E1FE01218807D5
:1024E000FFF76CFA012211469007FEF7BCFF0021AE
:1024F0004FF08040FFF730FA01218807FEF798FF80
:1025000007B000BD00B587B001210420FEF709FB2C
:1025100001210820FEF7F8FAC020ADF800000420E1
:102520008DF8030069463F48FEF732F804A8FEF72D
:102530004FFF0020ADF810004EF66020ADF81400FB
:102540004FF40070ADF816000020ADF8120004A999
:102550003748FEF711FC00231A4603213448FFF7E1
:102560001AF801A8FEF747FF0A20ADF80C0001A9F0
:102570002F48FEF794FE01212D48FFF71FFA012294
:1025800011462B48FEF76FFF00212948FFF7E4F9B9
:1025900001212748FEF74CFF07B000BD0146022984
:1025A00004D003290CD004291ED113E04FF080423F
:1025B000928C10B247F230524FF080439A8415E06B
:1025C000174A2432128810B247F23052144B243387
:1025D0001A800BE0164A2432128810B247F23052A9
:1025E000134B24331A8001E0002000BF00BF704766
:1025F0000F48103000880E481030008820F001008D
:102600000B491031088070474FF08040008A4FF02E
:102610008040008A20F001004FF08041088270471E
:1026200000040040000C0140001000400008014080
:102630000008004003461846884200DD08469042E4
:1026400000DA1046704770B50546A649284605F0E1
:1026500003FB04D3A449284605F0FEFB01D2012464
:1026600000E00024204670BD2DE9FE4F04460D46D3
:102670009E4E9F4F0021204605F01FFC02902946E8
:10268000002005F025FC01903946019805F018FB63
:1026900086F0004B00905846029905F011FB8246E7
:1026A000009905F015FC814605F06EFA804640461B
:1026B000BDE8FE8F10B501F065F88E4800688E49C0
:1026C00008608E49B1F9000005F09AFA8C4908605B
:1026D00010BD10B501218B48FFF767F9002852D0D3
:1026E00001218848FFF77EF90520FFF7C7FB02208C
:1026F000FFF754FF47F23051081A8349086004205D
:10270000FFF74CFF47F23051081A80490860FFF785
:10271000D1FF7E4803687C487DA10268844800F0B0
:10272000FBF97748016874480068FFF79DFF81490D
:10273000086071480068FFF786FF30B100F02EFB9B
:102740007DA17B4800F0E8F910BD7A4800687C491B
:10275000096808447B490860764800687849096838
:10276000084479490860794A514276480068FFF781
:1027700061FF74490860754A514273480068FFF769
:1027800059FF7149086000BFDEE72DE9FF5F04468D
:1027900089466F4803906F48029004EB0901484254
:1027A00005F02EFA6C4908606C48006805F05CF88A
:1027B00007466B4A6B4B04F063FE054604F026FCAB
:1027C000664908606448006805F04EF8644A664B44
:1027D000CDE9000104F054FE05460E465F4800684E
:1027E00005F042F807462A46334604F041FC82468B
:1027F00004F00CFC59490860084601685B48006811
:1028000005F05EF85949086059495848006805F0D4
:1028100023FB02D256485549086056495348006880
:1028200005F01AFA02D25348504908604F480299FD
:10283000006805F045FA07464848006880F0004601
:102840003046039905F03CFA0546394605F040FB51
:102850004949086028480068FFF7F5FE012803D0C1
:1028600046480078012802D10020404908604248CB
:10287000006805F089F904B0BDE8F09F0146002921
:1028800001DA484200E00846704770B505460C463C
:10289000002D03DD002000F01DFA02E0012000F011
:1028A00019FA2846FFF7EAFF35490880002C03DDB6
:1028B000002000F031FA02E0012000F02DFA20465D
:1028C000FFF7DCFF2E49091D088070BD012807D1E4
:1028D0002A49097809B9012100E00021274A11702D
:1028E00070470000000020C2000020420000C842E3
:1028F000713D8A3FC800002078000020B40000200D
:102900007C00002000100040400000204400002017
:10291000456E636F646572204C656674203D2025AA
:1029200064205269676874203D2025640D0A000008
:10293000004400408400002053746F700A000000BF
:10294000880000208C0000209000002094F8FFFFF9
:1029500000002043CDCC4C3F9C000020A000002074
:102960009A9999999999E93F9999C93FA4000020AA
:1029700000401C4600401CC698000020800000203B
:102980003C04004010B586B0044601210420FEF747
:10299000BBF801214804FEF7C4F80420ADF8140088
:1029A00018208DF8170003208DF8160005A9BA48E5
:1029B000FDF7EEFD0820ADF8140004208DF8170097
:1029C00005A9B548FDF7E4FD01940020ADF8080025
:1029D000ADF80A00ADF80C00ADF810000C20ADF811
:1029E0000E0001A9AD48FFF744F84FF4E060FDF791
:1029F00001FD26208DF8000000208DF801008DF8E3
:102A0000020001208DF803006846FDF7F8FC012262
:102A100040F22551A148FFF7C4F801219F48FFF774
:102A2000B4F806B010BD70B504460D4640219B4871
:102A3000FFF793F980219948FFF7C2F913E0217855
:102A40009648FFF70FF900BF40219448FFF778F947
:102A50000128F9D140219148FFF77FF980218F4863
:102A6000FFF7AEF9641C281EA5F10105E7D170BD82
:102A700010B5044640218948FFF76FF98021874847
:102A8000FFF79EF913E014F8011B8448FFF7EAF8FA
:102A900000BF40218148FFF753F90128F9D14021B7
:102AA0007E48FFF75AF980217C48FFF789F92078A2
:102AB0000028E8D110BDF0B503460D4616460027A4
:102AC00029460A2E03D0002008702846F0BD33B9ED
:102AD000302001F8010B002008702846F6E7002B93
:102AE00003DA2D2001F8010B5B4242F210720DE077
:102AF00093FBF2F404B937B104F1300001F8010B93
:102B000004FB123301270A2092FBF0F2002AEFDCCB
:102B1000002008702846D9E70FB470B586B0064685
:102B20000CA8009040215D48FFF717F980215B4811
:102B3000FFF746F97BE00B9800785C281CD10B98D6
:102B4000401C0B9000786E2809D072280FD10D21FF
:102B50003046FFF787F80B98401C0B900BE00A21DA
:102B60003046FFF77FF80B98401C0B9003E00B9862
:102B7000401C0B9000BF4BE00B980078252840D1FB
:102B80000B98401C0B900078642818D0732833D120
:102B9000009810C800900BE021783046FFF762F8EB
:102BA00000BF40213046FFF7CBF80028F9D0641C65
:102BB00020780028F0D10B98401C0B9020E0009862
:102BC00020C800900A2201A92846FFF774FF01AC33
:102BD0000BE021783046FFF745F800BF4021304632
:102BE000FFF7AEF80028F9D0641C20780028F0D157
:102BF0000B98401C0B9003E00B98401C0B9000BFFF
:102C000006E00B9810F8011B0B903046FFF72AF8EE
:102C100000BF40213046FFF793F80028F9D040214B
:102C20001E48FFF79AF880211C48FFF7C9F80B9857
:102C3000007800287FF47FAF06B070BC5DF814FB0D
:102C40000022174B1A60174A1160174A106070472C
:102C500010B540F225511148FFF788F8D8B10F4858
:102C6000FFF704F8C4B20F4800680D4909688842AC
:102C70000CD90D48006804700B480068401C0A49D4
:102C8000086007480068401C0549086040F225516B
:102C90000248FFF795F810BD0008014000440040CD
:102CA000AC000020B0000020A800002008B50121E1
:102CB0000820FDF729FF4FF47C40ADF800001020FC
:102CC0008DF8030003208DF8020069463748FDF7B0
:102CD0005FFC08BD10B504464CB94FF48051334831
:102CE000FDF703FD4FF400513048FDF700FD012CC6
:102CF00007D161032D48FDF7F8FC21032B48FDF7B0
:102D0000F6FC022C07D1E1022848FDF7F0FC210374
:102D10002648FDF7ECFC10BD10B504464CB94FF445
:102D200000412248FDF7E1FC4FF480411F48FDF7C8
:102D3000DEFC012C07D1A1031C48FDF7D6FCE10302
:102D40001A48FDF7D4FC022C07D161031748FDF7A0
:102D5000CEFCA1031548FDF7CAFC10BD10B500203C
:102D6000FFF7B8FF0020FFF7D7FF10BD10B5012017
:102D7000FFF7B0FF0120FFF7CFFF10BD10B5012016
:102D8000FFF7A8FF0020FFF7C7FF10BD10B5002018
:102D9000FFF7A0FF0120FFF7BFFF10BD10B5022015
:102DA000FFF798FF0220FFF7B7FF10BD000C0140AE
:102DB00008B501210820FDF7A7FE4FF44060ADF8EB
:102DC000000010208DF8030003208DF802006946F2
:102DD000F748FDF7DDFB08BD10B5F548001D00689C
:102DE00020F47040F249091D08600846006840F46C
:102DF000405008600120EF490860EF48D0F82C01EE
:102E000008B9002010BD0120EA49091F0860FFF73A
:102E100041F90020E849C1F8AC01E6488038006873
:102E200008B10020EEE70120FFF734F90020E14966
:102E3000091F08600120E5E710B5DD48001D0068A6
:102E400020F47040DA49091D08600846006840F423
:102E5000405008600020D749091F0860D649C1F8D2
:102E6000AC010120FFF716F90120D249091F0860C3
:102E7000D149C1F8AC01FFF70DF910BD10B5002420
:102E8000CB48001D006820F47040C949091D086046
:102E90000846006840F4004008600120C549086009
:102EA000FFF7F8F80120C449C1F8A801FFF7F2F8CC
:102EB0000AE0601CC4B2322C03DDFFF7BDFF002026
:102EC00010BD0120FFF7E6F8BA48803800680028F6
:102ED000EFD1B849091F08600120F1E710B50020C3
:102EE000B449091F0860B248001D006820F4704012
:102EF000AF49091D08600846006840F4405008606A
:102F00000020AD49C1F8AC010120FFF7C3F8012052
:102F1000A849091F0860FFF7BDF80020A649C1F8BD
:102F2000A80110BD10B50020A249091F0860A048E3
:102F3000001D006820F470409D49091D0860084686
:102F4000006840F44050086001209B49C1F8AC0182
:102F5000FFF7A0F801209749091F0860FFF79AF8CA
:102F600000209549C1F8A80110BD70B504469048ED
:102F7000001D006820F470408D49091D0860084656
:102F8000006840F44050086000208A49091F08602A
:102F9000002516E0E009874908606006040E01205C
:102FA000FFF778F801208449C1F8A801FFF772F80B
:102FB00000208049091F08600120FFF76BF8681C9A
:102FC000C5B2082DE6DB70BD2DE9F04105460E4681
:102FD00017469846FFF700FF10B90120BDE8F081C1
:102FE0006906080EFFF7C1FFFFF748FF18B9FFF7A2
:102FF00023FF0120F2E73046FFF7B7FFFFF73EFF60
:1030000000240BE018F80400FFF7AFFFFFF736FFCE
:1030100018B9FFF711FF0020E0E7641CBC42F1DBA8
:10302000FFF70AFF0020D9E770B505460024604885
:10303000001D006820F470405D49091D08600846C5
:10304000006840F400400860002617E0002059495D
:10305000091F08600220FFF71DF801205649C1F83A
:10306000A8016006040E53488038006808B1601C4F
:10307000C4B20220FFF70EF8701CC6B2082EE5DBC2
:1030800015B1FFF72BFF01E0FFF74CFF204670BDA5
:103090002DE9F04106460F4614461D46FFF79CFEFB
:1030A00010B90120BDE8F0817106080EFFF75DFF41
:1030B000FFF7E4FE18B9FFF7BFFE0120F2E738463C
:1030C000FFF753FFFFF7DAFEFFF786FE012101EB62
:1030D0004601C8B2FFF749FFFFF7D0FE0DE0012C13
:1030E00004D10020FFF7A0FF287003E00120FFF7C4
:1030F0009BFF28706D1C601EC4B2002CEFD1FFF73F
:103100009BFE0020CEE770B505460E460024FFF773
:1031100063FE2846FFF729FF641CFFF7AFFE304629
:10312000FFF723FF641CFFF7A9FEFFF755FE691C9C
:10313000C8B2FFF71AFF641CFFF7A0FE0020FFF7DC
:1031400073FF0446FFF778FE204670BD2DE9F0417D
:103150000746884615461E460024FFF73DFE3846C2
:10316000FFF703FFFFF78AFE4046FFF7FEFEFFF77B
:1031700085FEFFF731FE791CC8B2FFF7F6FEFFF7B8
:103180007DFE00BF0DE0681EA04204D00120FFF7C5
:103190004BFF305503E00020FFF746FF3055601C21
:1031A000C4B2AC42EFDBFFF747FE2046BDE8F0813A
:1031B000000C0140AC812142008021422DE9F04108
:1031C00080460D4616461F460024FFF705FE404682
:1031D000FFF7CBFEFFF752FE2846FFF7C6FEFFF7CC
:1031E0004DFE00BF06E0385DFFF7BFFEFFF746FE6D
:1031F000601CC4B2B442F6DBFFF71EFE0120BDE83E
:10320000F08170B505460E46144631462846FFF754
:103210007AFF2070012070BD37B504460D4602AB21
:10322000012229462046FFF7C9FF3EBD2DE9F8439C
:103230000746884614461D46089E6A46414638465B
:10324000FFF7DFFF28B3601CFF2101FA00F0C4F193
:1032500008012944491EFF220A41104300F0FF09DA
:10326000C5F1080006FA00F0C6B2C4F10700064135
:103270009DF8000000EA090000909DF8000030432E
:1032800000909DF8002041463846FFF7C5FFBDE895
:10329000F8830020FBE7F8B506460F4614461D46A6
:1032A0006A4639463046FFF7ACFF2DB10120A040F9
:1032B0009DF80010084305E00120A0409DF8001093
:1032C00021EA0000C0B200909DF800203946304647
:1032D000FFF7A2FFF8BD0000014691F90020002A87
:1032E00001DD00201EE091F90020002A01DA04200F
:1032F00018E091F90120002A01DD012012E091F986
:103300000120002A01DA05200CE091F90220002AB0
:1033100001DD022006E091F90220002A01DA0620F0
:1033200000E00720704770B505462846FFF7D4FF38
:103330000446E81CFFF7D0FF44EAC00084B2A81D91
:10334000FFF7CAFF44EA801084B2204670BD70B512
:1033500088B0F3A1F748FFF7DFFB02A905A801F049
:1033600092FF0446072C41D101A801F0FDF9059810
:1033700004F046FC0646019904F0A2FC054604F060
:1033800003FC0590069804F03BFC0646019904F006
:1033900097FC054604F0F8FB0690079804F030FC13
:1033A0000646019904F08CFC054604F0EDFB0790FD
:1033B00005A802F0A2FA684601F0F3F9BDF8001082
:1033C000029848430290BDF80010039848430390C8
:1033D000BDF8001004984843049002A802F020FBB6
:1033E0002246D5A1D348FFF797FB04E02246DBA194
:1033F000D048FFF791FB08B070BD2DE9F0430446BB
:103400000D46DDE907670021012041E0DFF858C3E0
:103410003CF81080A0F1010CDFF84C9329F81C80D7
:1034200009F1160C3CF81090A0F1010CDFF838837C
:1034300008F1160828F81C9008F1160C3CF81090BA
:10344000A0F1010C08F1160828F81C9008F1160CE0
:103450003CF81090A0F1010C08F1160828F81C9017
:1034600008F1160C3CF81090A0F1010C08F11608B8
:1034700028F81C9008F1160C3CF81090A0F1010CF3
:1034800008F1160828F81C9000F1010C0CF0FF0060
:103490000A28BBDBDFF8D0C2ACF81240ACF82850E9
:1034A000ACF83E20ACF85430ACF86A60ACF88070F0
:1034B0000021002008E0DFF8B0C23CF910C06144F0
:1034C00000F1010C0CF0FF000A28F4DB4FF00A0CAD
:1034D00091FBFCFC0FFA8CFCDFF88C82A8F814C07E
:1034E000002100200AE0DFF880C20CF1160C3CF944
:1034F00010C0614400F1010C0CF0FF000A28F2DB5F
:103500004FF00A0C91FBFCFC0FFA8CF8DFF858C264
:10351000ACF82A80002100200AE0DFF84CC20CF150
:103520002C0C3CF910C0614400F1010C0CF0FF00C0
:103530000A28F2DB4FF00A0C91FBFCFC0FFA8CF826
:10354000DFF824C2ACF84080002100200AE0DFF858
:1035500018C20CF1420C3CF910C0614400F1010C9E
:103560000CF0FF000A28F2DB4FF00A0C91FBFCFC88
:103570000FFA8CF8DFF8F0C1ACF85680002100207B
:103580000AE0DFF8E4C10CF1580C3CF910C06144CA
:1035900000F1010C0CF0FF000A28F2DB4FF00A0CDE
:1035A00091FBFCFC0FFA8CF8DFF8BCC1ACF86C8026
:1035B000002100200AE0DFF8B0C10CF16E0C3CF9EC
:1035C00010C0614400F1010C0CF0FF000A28F2DB8E
:1035D0004FF00A0C91FBFCFC0FFA8CF8DFF888C165
:1035E000ACF88280BDE8F08338B50446032302229C
:1035F0006B21D0200094FFF719FE38BD38B5044682
:10360000022304221B21D0200094FFF70FFE38BDB7
:1036100038B50446022304221C21D0200094FFF771
:1036200005FE38BD10B50446234606226B21D02086
:10363000FFF731FE10BD10B54C4B01227521D02093
:10364000FFF784FD4948007810BD10B5FFF7F3FF80
:10365000682801D1012010BD0020FCE710B5044608
:10366000234605226A21D020FFF715FE10BD10B5B4
:103670000446234601223721D020FFF70CFE10BD5F
:1036800010B50220FFF7B0FF0320FFF7B7FF0020BF
:10369000FFF7BEFF0020FFF7C5FF0020FFF7DEFFAA
:1036A0000020FFF7E4FF10BD38B5002000906B4606
:1036B000012275216820FFF7EBFC9DF800006828C7
:1036C00006D09DF800202AA11A48FFF725FA05E048
:1036D0009DF8002026A11748FFF71EFA00F051FDC3
:1036E000E0B9782000F0B5F9782000F099FBC82007
:1036F00000F077FC02F066F82148FFF714FE04465C
:1037000002F06AF840F2731002F0A7FCC82002F041
:103710001DFAFFF71CFE012001F06CFD38BD000012
:1037200072756E5F73656C665F746573742E2E0DB3
:103730000A0000000044004073657474696E6720DD
:10374000626961732073756363657366756C6C7908
:10375000202E2E2E2564200D0A0000004661696C83
:103760002E2E2025640D0A002601002018010020BD
:1037700077686F20616D20692025640D0A000000C4
:10378000DC0000202DE9F04F8DB00AA849490BABB1
:1037900006AACDE900104849484802F0BDFD454859
:1037A000008800F4807000287ED0069804F028FA83
:1037B00004464FF09D4104F0F1F841490860079834
:1037C00004F01EFA04464FF09D4104F0E7F83D492D
:1037D0000860089804F014FA04464FF09D4104F084
:1037E000DDF839490860099804F00AFA04464FF0F8
:1037F0009D4104F0D3F835490860334801684FF023
:10380000804004F05DFA01902F480168019804F0AF
:1038100057FA82462B4801684FF0404004F050FAB6
:10382000019028480168019804F04AFA83465146FD
:1038300004F04EFB81464FF07E5104F041F80446FF
:1038400004F012F8CDE902011D4801684FF08040F4
:1038500004F036FA83461B480168584604F030FAF3
:103860008146194801684FF0804004F029FA8346E8
:1038700016480168584604F023FA8246494604F087
:103880001FF8044603F0F0FF0746DDE9022303F0CA
:10389000FDFA4FF066320E4BCDE9040103F0F0FD66
:1038A000054603F0B3FB00E001E00A4908600DB0F3
:1038B000BDE8F08FC0000020BA000020B400002056
:1038C000CC000020D0000020D4000020D800002030
:1038D00066A64C40C800002038B50446FB4890F866
:1038E0002400C0B114B10220009001E0002000903B
:1038F000F64A1268D17BF54A526810786B4601226D
:10390000FFF762FB10B14FF0FF3038BD9DF800109B
:10391000EE48417423E0ED48807A10B94FF0FF3053
:10392000F3E724B1E948407C08B10020EDE714B189
:103930000120009001E000200090E44A1268D17B51
:10394000E24A526810786B460122FFF73DFB10B146
:103950004FF0FF30D9E79DF80010DC48417400209B
:10396000D3E738B5002419E0D8480068C07AA042EF
:1039700004D0D6480068407DA04200D10CE0D34975
:10398000496808786B4601222146FFF781FB10B198
:103990004FF0FF3038BD00BF601CC4B2CB48406858
:1039A0000079A042E0DC0020F4E770B504460D4643
:1039B000C6480068C07AA04204D0C4480068407D70
:1039C000A04202D14FF0FF3070BDC048406800797E
:1039D000A04202DC4FF0FF30F6E7BC4949680878A6
:1039E0002B4601222146FFF753FBEDE738B504468D
:1039F000B64890F82300A04201D1002038BD14B190
:103A00003020009001E000200090B048807C20B180
:103A10009DF8000040F002000090AC4890F82200B1
:103A200020B19DF8000040F080000090A74A126885
:103A3000117DA64A526810786B460122FFF7C4FA3E
:103A400010B14FF0FF30D9E7A04880F823400020A4
:103A5000D4E738B5044604F0700010B1012000909E
:103A600005E014B10020009001E040200090974A4A
:103A70001268917C954A526810786B460122FFF7D4
:103A8000A3FA20B1002191488172481E38BD9DF8EB
:103A9000000020F040018D4801730020009004F0E8
:103AA000400020B99DF8000040F00400009004F0B0
:103AB000200020B99DF8000040F00200009004F0C2
:103AC000100020B99DF8000040F00100009004F0C3
:103AD000080020B99DF8000040F0380000907B4AB3
:103AE0001268D17C794A526810786B460122FFF740
:103AF0006BFA20B1002175488172481EC6E724B1D7
:103B0000082C02D00020FFF771FF7048847200215A
:103B100001753220FEF7A2FA0020B7E738B5044657
:103B20006A48807CA04201D1002038BD002C46D0DC
:103B3000664A12681179654A526810786B4601220C
:103B4000FFF7A6FA10B14FF0FF30EEE79DF8000046
:103B500020F0200000905D4A126811795B4A52689B
:103B600010786B460122FFF72FFA10B14FF0FF30AB
:103B7000DBE70320FEF772FA02200090534890F82A
:103B8000220020B19DF8000040F0800000904F48D6
:103B900090F8230020B19DF8000040F03000009024
:103BA0004A4A1268117D494A526810786B460122D0
:103BB000FFF70AFA002851D04FF0FF30B5E7434A2B
:103BC00012681179414A526810786B460122FFF75A
:103BD0005FFA10B14FF0FF30A7E73C48807A00F061
:103BE000010028B19DF8000040F02000009004E0A2
:103BF0009DF8000020F020000090344A12681179EE
:103C0000324A526810786B460122FFF7DDF910B195
:103C10004FF0FF3089E70320FEF720FA2B4890F899
:103C2000220010B18020009001E000200090274881
:103C300090F8230020B19DF8000040F03000009083
:103C4000224A1268117D214A526810786B4601227F
:103C5000FFF7BAF910B14FF0FF3066E71B488474E4
:103C6000002062E708B51948807A10B94FF0FF309C
:103C700008BD00200090154A1268D17B134A526893
:103C800010786B460122FFF79FF910B14FF0FF301B
:103C9000EEE70E4A126851790C4A526810786B466A
:103CA0000122FFF791F910B14FF0FF30E0E7074A2A
:103CB00012681179054A526810786B460122FFF7A5
:103CC00083F928B14FF0FF30D2E70000EC0000206C
:103CD000F74890F82400002850D00C200090F44AB7
:103CE00012681179F24A526810786B460122FFF788
:103CF0006BF910B14FF0FF30BAE7C0200090EC48EC
:103D0000807A00F0010020B19DF8000040F0200012
:103D10000090E74A12681179E54A526810786B46BC
:103D20000122FFF751F910B14FF0FF30A0E7E04852
:103D3000407C10B10220009001E000200090DC4A9D
:103D40001268D17BDA4A526810786B460122FFF77D
:103D50003BF910B14FF0FF308AE700200090D44AC1
:103D600012685179D24A526810786B460122FFF7E7
:103D70002BF9002852D04FF0FF3079E70420009053
:103D8000CB4A12681179CA4A526810786B460122F0
:103D9000FFF71AF910B14FF0FF3069E7C448807C93
:103DA00020B9C348807A00F0010010B9402000908B
:103DB00001E060200090BE4A12681179BC4A526846
:103DC00010786B460122FFF7FFF810B14FF0FF307B
:103DD0004EE7B748407C10B10120009001E0002080
:103DE0000090B34A1268D17BB14A526810786B4692
:103DF0000122FFF7E9F810B14FF0FF3038E7AC4A85
:103E000012685179AA4A52681078A94B10330122DE
:103E1000FFF7DAF810B14FF0FF3029E7002027E76D
:103E200070B50446002624F00104A14890F824004F
:103E300008B1002070BD9E48807A10B94FF0FF3065
:103E4000F8E79B48057C807A204099490874084629
:103E5000007CA04202D04FF0FF3600E0002614B9EB
:103E60009348007D18B10120FFF736FD02E00020E5
:103E7000FFF732FD3CB1FFF7F5FE20B18C48057429
:103E80004FF0FF30D6E73046D4E738B504468848CF
:103E9000807A10B94FF0FF3038BDBC2C02DB012016
:103EA000009015E0622C02DB0220009010E02A2C2A
:103EB00002DB032000900BE0142C02DB04200090B6
:103EC00006E00A2C02DB0520009001E006200090AD
:103ED0007748C07A9DF80010884201D10020DBE7C6
:103EE000734A12689178724A526810786B460122C0
:103EF000FFF76AF810B14FF0FF30CDE79DF80010E2
:103F00006B48C1720020C7E738B50446282C02DD93
:103F10004FF0FF3038BDDCB90020FFF767FD00200F
:103F20008DF8000007208DF80100614A1268917C2D
:103F30005F4A526810786B460222FFF745F810B1CD
:103F40004FF0FF30E6E70021594801750020E1E716
:103F50000120FFF74BFD20208DF80000012C06D139
:103F600000208DF801000520FFF78FFF17E0052CDA
:103F700006DC01208DF801000520FFF786FF0EE02A
:103F8000142C06DC02208DF801000A20FFF77DFFCB
:103F900005E003208DF801001420FFF776FF9DF85F
:103FA0000100072101EB8010C0B28DF80100404AEA
:103FB0001268917C3E4A526810786B460222FFF7E5
:103FC00003F810B14FF0FF30A4E7082138488172A0
:103FD00000210173012101750020FFF721FF00205E
:103FE00098E738B504463248807A10B94FF0FF3070
:103FF00038BD2F4890F8240010B14FF0FF30F7E79C
:104000002B48007D50B134B1282C04DCE0B2FFF71E
:104010007BFF0020ECE70020FFF776FF042C01DA9D
:10402000042404E0B4F57A7F01DD4FF47A744FF490
:104030007A7090FBF4F0401EC0B200901C4A1268E7
:1040400051781B4A526810786B460122FEF7BCFF7C
:1040500010B14FF0FF30CBE79DF80000401C4FF44B
:104060007A7191FBF0F081B21148C1810146C98992
:104070004810FFF70AFF0020BAE738B504460C489D
:10408000807A10B94FF0FF3038BD022C06D0042CD6
:1040900007D0082C08D0102C0FD10BE00020009086
:1040A0000EE0082000900BE01020009008E00000D7
:1040B000EC0000201820009002E04FF0FF30E3E712
:1040C00000BFF948407A9DF80010B0EBE10F01D134
:1040D0000020D9E7F44A1268D179F34A526810787F
:1040E0006B460122FEF770FF10B14FF0FF30CBE7B7
:1040F0009DF80000C110EC4841720020C4E738B5BB
:104100000446E948807A10B94FF0FF3038BDFA2CE8
:1041100009D0B4F5FA7F09D0B4F57A7F09D0B4F5A7
:10412000FA6F0CD108E0002000900BE0082000900E
:1041300008E01020009005E01820009002E04FF009
:10414000FF30E3E700BFD848007A9DF80010B0EBDD
:10415000E10F01D10020D9E7D34A12689179D24A00
:10416000526810786B460122FEF72EFF10B14FF017
:10417000FF30CBE79DF80000C010CB49087200204B
:10418000C4E71CB580208DF80000C74A1268917CF6
:10419000C54A526810786B460122FEF715FF10B130
:1041A0004FF0FF301CBD6420FDF758FF00208DF854
:1041B0000000BD4A1268917CBB4A526810786B4679
:1041C0000122FEF701FF10B14FF0FF30EAE7B64AD7
:1041D0001268917DB44A526810786B460622FEF749
:1041E00057FF10B14FF0FF30DCE79DF80500C00726
:1041F000400F9DF8031001F0010140EA41009DF8D5
:10420000011001F0010140EA010494B1012C03D135
:104210000121A548C17431E0022C03D10021A2483C
:10422000C1742BE02146A1A002F07CFA4FF0FF30D0
:10423000B8E79D4A1268D1789B4A526810786B465D
:104240000122FEF725FF10B14FF0FF30AAE79DF8DD
:10425000000000F00F042CB99E4802F063FA4FF002
:10426000FF309FE7042C06D19BA002F05BFA0121EE
:104270008D48C17402E000218B48C174FF218A4837
:104280008172FF2088490872FF2187484172C172FC
:104290004FF6FF71C181FF21017481740121017307
:1042A00080F82210002180F8231041750175163026
:1042B000016041608160163880F8241080F8251074
:1042C000C1844FF4FA60FFF71AFF10B14FF0FF30CE
:1042D00068E70220FFF7D1FE10B14FF0FF3061E731
:1042E0002A20FFF7D2FD10B14FF0FF305AE73220FD
:1042F000FFF777FE10B14FF0FF3053E70020FFF7D4
:104300008FFD10B14FF0FF304CE70020FFF706FCA7
:1043100010B14FF0FF3045E70020FFF79AFB002077
:1043200040E770477CB504460D465F48807A00F050
:10433000700010B94FF0FF307CBD5B4A1268117BF2
:10434000594A526810786B460622FEF7A1FE10B15A
:104350004FF0FF30F0E79DF801009DF8001040EAB3
:10436000012000B220809DF803009DF8021040EA71
:10437000012000B260809DF805009DF8041040EA1D
:10438000012000B2A08015B12846FFF7CAFF002027
:10439000D2E77CB504460D464348807A00F0080019
:1043A00010B94FF0FF307CBD3F4A1268517B3E4A46
:1043B000526810786B460622FEF76AFE10B14FF085
:1043C000FF30F0E79DF801009DF8001040EA012061
:1043D00000B220809DF803009DF8021040EA012001
:1043E00000B260809DF805009DF8041040EA0120AD
:1043F00000B2A08015B12846FFF793FF0020D2E756
:104400002DE9FE4F05460C462748807A18B94FF033
:10441000FF30BDE8FE8F244A1268917B224A526821
:10442000107802AB0222FEF733FE10B14FF0FF30DE
:10443000EFE79DF809009DF8081040EA012006B258
:1044400014B12046FFF76DFF17494968C88803F08B
:10445000EFFB154901904968B1F9080003F0D0FB62
:104460008346304603F0CCFB5946009003F030FD04
:104470008246019903F092FA81461F4903F020FA1F
:1044800080464FF08F4103F01BFC074603F07CFB96
:1044900028600020BDE710B588B004461CB94FF075
:1044A000FF3008B010BD29E0EC000020556E737598
:1044B00070706F7274656420736F66747761726573
:1044C0002070726F64756374207265762025642E87
:1044D0000A000000988D000848616C662073656EC4
:1044E0007369746976697479207061727420666F7B
:1044F000756E642E0D0A000000000C42206830B971
:10450000606820B9A06810B9002008B010BDFA4951
:104510004968087806AB03221146FEF7B9FD10B1D1
:104520004FF0FF30F1E79DF81800082101EB201053
:1045300000F00F00ADF800009DF8190001EB20100D
:1045400000F00F00ADF802009DF81A0001EB2010FA
:1045500000F00F00ADF8040020684100BDF9000034
:10456000403091FBF0F000B2ADF8100060684100FF
:10457000BDF90200403091FBF0F000B2ADF812003E
:10458000A0684100BDF90400403091FBF0F000B29A
:10459000ADF81400D8494968087806AB06221146E0
:1045A000FEF776FD10B14FF0FF30AEE79DF8190031
:1045B0009DF8181040EA012000B2ADF808009DF8FF
:1045C0001B009DF81A1040EA012000B2ADF80A0065
:1045D0009DF81D009DF81C1040EA012000B2ADF8C6
:1045E0000C00BDF81000BDF80810084400B2ADF88A
:1045F0001000BDF81200BDF80A10084400B2ADF872
:104600001200BDF81400BDF80C10084400B2ADF85B
:104610001400BDF81000000A8DF81800BDF8100055
:10462000C0B28DF81900BDF81200000A8DF81A000A
:10463000BDF81200C0B28DF81B00BDF81400000ACE
:104640008DF81C00BDF81400C0B28DF81D00AA49F9
:104650004968087806AB06221146FEF7B5FC10B192
:104660004FF0FF3051E700204FE70146A248007AA3
:1046700030B1012807D0022809D003280FD10AE061
:10468000FA2008800EE04FF4FA7008800AE04FF438
:104690007A70088006E04FF4FA60088002E000209B
:1046A000088000BF00BF0020704701469248407A52
:1046B00030B1012807D0022808D003280CD108E027
:1046C000022008700BE00420087008E00820087041
:1046D00005E01020087002E04FF0FF30704700BF87
:1046E0008548C07C18B108784006000E087000208C
:1046F000F4E701468048C07A082817D2DFE800F0C6
:104700001704070A0D101318BC20088013E062205C
:10471000088010E02A2008800DE0142008800AE0BC
:104720000A20088007E00520088004E000BF00BFE1
:104730000020088000BF00BF0020704701466E487F
:1047400090F8240010B14FF0FF3070476A48C089DC
:1047500008800020F9E7014600200880401E7047CD
:1047600001464FF0FF30704701466348007A30B190
:10477000012807D0022808D003280CD108E05F48A0
:1047800008600BE05E48086008E05E48086005E0ED
:104790005D48086002E04FF0FF30704700BF002026
:1047A000FBE701465448407A30B1012808D002287E
:1047B0000AD0032810D10BE04FF4804008800EE0AF
:1047C00041F69C7008800AE04FF48050088006E0B3
:1047D0004FF40060088002E04FF0FF30704700BFE8
:1047E0004548C07C10B10888401008800020F5E7DB
:1047F00001464148007C08700020704701463E4851
:10480000807A10B10120087001E0002008700020BB
:10481000704738B504463848807A10B94FF0FF30F9
:1048200038BD354A1268117C334A526810786B469D
:104830000222FEF72DFC10B14FF0FF30F0E79DF89B
:1048400001009DF8001040EA012000B22080002005
:10485000E6E72DE9FE4F0746884692461D46DDF8FD
:1048600030B000260024244890F8240010B1601EC7
:10487000BDE8FE8F002028701F48807A10B94FF0E5
:10488000FF30F5E71C48007C10B94FF0FF30EFE730
:104890001948007C00F0400008B1B01CC6B21648B0
:1048A000007C00F0200008B1B01CC6B21248007CA9
:1048B00000F0100008B1B01CC6B20F48007C00F038
:1048C000080008B1B01DC6B20B4A1268917A0A4AB4
:1048D000526810786B460222FEF7DAFB10B14FF0F7
:1048E000FF30C5E79DF801009DF8001040EA01295E
:1048F000B1450BDA0020BBE7EC00002000000343C9
:10490000000083423333034233338341FC48406821
:104910004088B9EB600F17DDF94A1268517CF84AFC
:10492000526810786B460122FEF7B2FB10B14FF0CF
:10493000FF309DE79DF8000000F0100020B1FFF768
:1049400091F96FF0010093E75046FFF7EAFCEC4A5B
:104950001268D17AEA4A526810786B463246FEF7FE
:1049600097FB10B14FF0FF3082E799FBF6F0401E45
:104970008BF8000000202870B4422AD0E048007C68
:1049800000F0080028B3601C1DF800001DF804109A
:1049900040EA012000B2A8F80000E01C1DF8001059
:1049A000A01C1DF8000041EA002000B2A8F8020097
:1049B000601D1DF80010201D1DF8000041EA0020B8
:1049C00000B2A8F80400287840F008002870A01D64
:1049D00084B2B44213D0CA48007C00F0400070B1E9
:1049E000601C1DF800001DF8041040EA012000B210
:1049F0003880287840F040002870A01C84B2B4426F
:104A000013D0BF48007C00F0200070B1601C1DF87E
:104A100000001DF8041040EA012000B278802878D8
:104A200040F020002870A01C84B2B44213D0B448D7
:104A3000007C00F0100070B1601C1DF800001DF833
:104A4000041040EA012000B2B880287840F010003D
:104A50002870A01C84B200200AE7F8B504460F466F
:104A60001646A74890F8240010B94FF0FF30F8BD63
:104A7000A348807A10B94FF0FF30F8E7A04A1268D7
:104A8000917A9F4A526810786B460222FEF700FB2B
:104A900010B14FF0FF30EAE79DF801009DF80010DB
:104AA00040EA0125A54203DA00203070401EDEE70F
:104AB000934840684088B5EB600F17DD904A126854
:104AC000517C8F4A526810786B460122FEF7E0FA5B
:104AD00010B14FF0FF30CAE79DF8000000F0100061
:104AE00020B1FFF7BFF86FF00100C0E7E2B2844BDE
:104AF0001B68D97A824B5B6818783B46FEF7C8FA88
:104B000010B14FF0FF30B2E795FBF4F0401E30706B
:104B10000020ACE701467A4880F822100020704758
:104B20007CB5054676494968087801AB04220D2119
:104B3000FEF7AEFA08B107207CBD9DF80700C0F370
:104B400001109DF8041001F0E00140EAE1008DF849
:104B500000009DF80700C0F381009DF8051001F0EA
:104B6000E00140EAE1008DF801009DF8070000F047
:104B700003009DF8061001F0E00140EAE1008DF825
:104B8000020000241CE01DF8040018B9002045F8BC
:104B9000240013E05B4845F8240006E055F82400A3
:104BA000594903F08DF845F824001DF80400401E13
:104BB000C0B20DF804000028F0D100BF601CC4B2E0
:104BC000032CE0DB0020B7E72DE9FE4F06460F4639
:104BD00000256846FFF7A4FF002442E056F82400B1
:104BE00057F82410A0EB010ABAF1000F01DB51467F
:104BF00001E0CAF10001084603F002F883464FF0D5
:104C00008F4102F0CBFE80465DF82400002102F0C7
:104C100087FF16D05DF82410404602F0BFFE8246A2
:104C20004FF07E5103F054F9814629F0004A37488D
:104C3000416A504603F010F912D20120A04005430A
:104C40000EE03248C169404603F006F805D32F480C
:104C5000016A404603F000F902D20120A04005435A
:104C6000641C032CBADB2846BDE8FE8F2DE9FC5FEF
:104C700006460F46002522494968087801AB032201
:104C80000D21FEF705FA10B10720BDE8FC9F9DF845
:104C9000040000F01F008DF804009DF8050000F0EE
:104CA0001F008DF805009DF8060000F01F008DF82C
:104CB0000600002462E056F8240057F82410A0EB08
:104CC000010BBBF1000F01DB594601E0CBF1000104
:104CD000084602F095FF4FF08F41009002F05EFE13
:104CE000814601A8005DC0B30849086802F0A0FF32
:104CF00083465946064802F051FE80460FE0000008
:104D0000EC0000207B14AE3E1D5A843FD480000886
:104D100000B04C45FE49404602F0D2FF804601A853
:104D2000005D401EC0B201A908550028F2D14146DD
:104D3000484602F033FE83464FF07E5103F0C8F838
:104D400082462AF0004BF3488169584603F084F804
:104D500013D20120A04005430FE0FFE7ED480169B1
:104D6000484602F079FF05D3EA484169484603F016
:104D700073F802D20120A0400543641C032C9ADB87
:104D8000284682E72DE9F04F87B005460C4691464C
:104D900001208DF8100000208DF81100DE4A126805
:104DA000917CDD4A5268107804AB0222FEF70CF9C0
:104DB00020B14FF0FF3007B0BDE8F08FC820FDF7FD
:104DC0004DF900208DF81000D34A1268D17BD24AE9
:104DD0005268107804AB0122FEF7F6F810B14FF0DC
:104DE000FF30E8E7CC4A12685179CB4A5268107814
:104DF00004AB0122FEF7E8F810B14FF0FF30DAE71C
:104E0000C54A1268917CC44A5268107804AB0122EA
:104E1000FEF7DAF810B14FF0FF30CCE7BE4A126867
:104E2000D17DBD4A5268107804AB0122FEF7CCF860
:104E300010B14FF0FF30BEE7B74A12681179B64A99
:104E40005268107804AB0122FEF7BEF810B14FF0A3
:104E5000FF30B0E70C208DF81000AF4A12681179CE
:104E6000AD4A5268107804AB0122FEF7ADF810B1DC
:104E70004FF0FF309FE70F20FDF7F0F8A648806A5B
:104E8000407A8DF81000A44A12689178A24A5268BC
:104E9000107804AB0122FEF797F810B14FF0FF3005
:104EA00089E79D48806A007A8DF810009A4A126856
:104EB0005178994A5268107804AB0122FEF784F8C1
:104EC00010B14FF0FF3076E7B9F1000F07D09248EC
:104ED000806A807A40F0E0008DF8100004E08E488F
:104EE000806A807A8DF810008B4A126891798A4A1C
:104EF0005268107804AB0122FEF766F810B14FF04B
:104F0000FF3058E7B9F1000F07D08348806AC07AB4
:104F100040F0E0008DF8100003E07E48C07A8DF884
:104F200010007D4A1268D1797B4A5268107804AB30
:104F30000122FEF749F810B14FF0FF303BE7B9F11D
:104F4000000F02D0C820FDF789F840208DF810002E
:104F5000714A12681179704A5268107804AB0122C4
:104F6000FEF732F810B14FF0FF3024E778208DF8CB
:104F70001000694A12685179674A5268107804AB88
:104F80000122FEF721F810B14FF0FF3013E761491D
:104F90008889FDF763F800208DF810005E4A1268DA
:104FA00051795D4A5268107804AB0122FEF70CF883
:104FB00010B14FF0FF30FEE6574A1268917A564A18
:104FC0005268107804AB0222FEF762F810B14FF07D
:104FD000FF30F0E69DF811009DF8101040EA012B1B
:104FE0000C209BFBF0F0C6B20020A860686028602F
:104FF000A06060602060824665E0474A1268D17A0E
:10500000454A5268107804AB0C22FEF741F810B103
:105010004FF0FF30CFE69DF811009DF8101040EAE8
:10502000012000B2ADF808009DF813009DF81210A1
:1050300040EA012000B2ADF80A009DF815009DF885
:10504000141040EA012000B2ADF80C00BDF90810C0
:10505000206808442060BDF90A1060680844606058
:10506000BDF90C10A0680844A0609DF817009DF8D9
:10507000161040EA012000B2ADF800009DF81900BA
:105080009DF8181040EA012000B2ADF802009DF82A
:105090001B009DF81A1040EA012000B2ADF8040090
:1050A000BDF90010286808442860BDF9021068683E
:1050B00008446860BDF90410A8680844A8600AF1B3
:1050C000010000F0FF0AB24597DB1248D0F800C09B
:1050D0002868C117090441EA104107046246002309
:1050E000384601F0FAFA32460023CDE9020101F018
:1050F000F4FA28600748D0F800C06868C1170904AE
:1051000041EA1041070462460023384606E00000E9
:1051100054E3853FD4800008EC00002001F0DDFA64
:1051200032460023CDE9020101F0D7FA6860F94860
:10513000D0F800C0A868C117090441EA104107046B
:1051400062460023384601F0C8FA32460023CDE912
:10515000020101F0C2FAA860EE48D0F804C021684C
:10516000C817000440EA11480F046246002338467D
:10517000414601F0B2FA32460023CDE9020101F0C6
:10518000ACFA2060E348D0F804C06068C117090495
:1051900041EA1041070462460023384601F09DFAB7
:1051A00032460023CDE9020101F097FA6060D94848
:1051B000D0F804C0A068C117090441EA10410704EF
:1051C00062460023384601F088FA32460023CDE9D2
:1051D000020101F082FAA060A068002804DDA06846
:1051E000A0F58030A06003E0A06800F58030A060EA
:1051F0000020E0E538B50446C74890F82400A042F6
:1052000001D1002038BD44B3C34890F8250010B93F
:105210004FF0FF30F6E70020FEF75EFB0020FEF7C0
:105220007DFCBD49C88CFEF7DCFE00200090BA4929
:10523000496808786B4601222321FDF7C5FE01214C
:10524000B54880F824100120FEF746FBFEF70AFD62
:10525000B2A1B948FDF760FC13E00020FEF73CFB6B
:10526000AD48007C0090AC49496808786B46012243
:105270002321FDF7A9FE0021A74880F82410FEF79E
:10528000F1FC0020BEE72DE9F04F8DB083460F46BC
:1052900002200C90A04890F8240020B10020FFF7D5
:1052A000A9FF012600E0002603A8FFF7DEF905A804
:1052B000FFF7FBF901A8FFF71CFA02A8FFF73EFA77
:1052C000954890F80AA004A8FFF792FA002407E096
:1052D000002239465846FFF755FD00B902E0641C2C
:1052E000022CF5DB00BF022C01D1002528E00024B0
:1052F00007E0012206A909A8FFF744FD00B902E072
:10530000641C022CF5DB00BF022C01D1002517E044
:1053100006A93846FFF758FC00F0FF0809A95846CF
:10532000FFF7A4FC00F0FF090025B9F1000F01D13F
:1053300045F00105B8F1000F01D145F0020500BFAD
:10534000FF2075490872FF2173484172C1724FF600
:10535000FF71C181FF218172017401210173BDF8C8
:105360000C00FEF7CCFE9DF81400FEF786FEBDF89B
:105370000400FEF78AFDBDF80800FEF732FE504635
:10538000FEF767FB9DF81000FEF74AFD3EB10120D5
:10539000FFF730FF2A4669A16748FDF7BDFB2A46A3
:1053A00069A16548FDF7B8FB28460DB0BDE8F08F50
:1053B000F8B504460D46164616B94FF0FF30F8BD55
:1053C0005548807A10B94FF0FF30F8E720128DF879
:1053D0000000E0B28DF801009DF8010028444E491C
:1053E00049684989884202DD4FF0FF30E7E74A4AC1
:1053F0001268117E484A526810786B460222FDF707
:10540000E3FD10B14FF0FF30D9E7EAB2424B1B6821
:10541000597D414B5B6818783346FDF7D5FD10B1D7
:105420004FF0FF30CBE70020C9E7F8B504460D4642
:10543000164616B94FF0FF30F8BD3748807A10B9DC
:105440004FF0FF30F8E720128DF80000E0B28DF841
:1054500001009DF8010028442F4949684989884284
:1054600002DD4FF0FF30E7E72B4A1268117E2A4A2F
:10547000526810786B460222FDF7A6FD10B14FF07E
:10548000FF30D9E7EAB2244B1B68597D224B5B6899
:1054900018783346FDF7FCFD10B14FF0FF30CBE735
:1054A0000020C9E72DE9F04385B005460E46904639
:1054B0009946194890F8250020B14FF0FF3005B00B
:1054C000BDE8F08316B94FF0FF30F8E7002447E05D
:1054D000281B102801DD102000E0281B87B232199C
:1054E00039462046FFF764FF10B14FF0FF30E6E782
:1054F00001AA39462046FFF798FF10B14FF0FF3060
:10550000DDE730193A4601A901F088F930B36FF0B0
:105510000100D4E7D4800008EC0000206D70755FB6
:105520007365745F646D705F737461746520646D1E
:1055300070206F6E0D0A000000440040646D702002
:105540006F6E0D0A0000000072657475726E2E2E6B
:10555000726573203D2025640D0A0000E01984B2B5
:10556000AC42B5DB4FEA28208DF8000008F0FF00C0
:105570008DF80100924A1268917E914A5268107823
:105580006B460222FDF720FD10B14FF0FF3096E789
:1055900001218B4880F82510A0F8269000208EE786
:1055A0000146874890F824000870002070470246A2
:1055B0004FF0FF30704701464FF0FF307047F8B5AD
:1055C00005460F461446002C70D0B5F5FF5F01DD8F
:1055D000FF2605E0202D01DA012601E0C5F347167C
:1055E00007B90127282C02DD4FF0FF30F8BD7448C1
:1055F000407D28BB724890F8240038B10020FFF7A6
:10560000F9FD01216E4880F8201003E000216C486C
:1056100080F820106A481630FFF727F868481830DD
:10562000FFF743F866481A30FFF763F864481C3008
:10563000FFF784F86248817A81771F30FFF7D8F846
:105640000020FEF749F90020FEF75EFC00208DF8EF
:1056500000005B4A12689178594A526810786B468C
:105660000122FDF7B1FC10B14FF0FF30BEE7402042
:105670008DF80000524A1268D17B514A5268107866
:105680006B460122FDF7A0FC00B165E08DF80060DB
:105690008DF801704A4A1268117A494A52681078A6
:1056A0006B460222FDF790FC08B155E047E005206B
:1056B000FCF7D4FC4248407A072101EBC000C0B29D
:1056C0008DF800003E4A1268D1793D4A5268107840
:1056D0006B460122FDF778FC00B13DE020208DF8FB
:1056E0000000012C03D100208DF801000EE0052CF4
:1056F00003DC01208DF8010008E0142C03DC0220FB
:105700008DF8010002E003208DF801009DF80100F2
:10571000072101EB8010C0B28DF80100284A126801
:10572000917C274A526810786B460222FDF74CFCA8
:1057300000B111E0012122484175002056E7204ABE
:105740001632002103E0505C00B105E0491C0C2931
:10575000F9D34FF0FF3049E7FF2019490872FF21C4
:1057600017484172C1724FF6FF71C181FF218172EA
:105770000174012101730146887FFEF76AF910491F
:10578000C88AFEF7BCFC0E49087EFEF776FC0C4981
:10579000488BFEF77AFB0A49888BFEF722FC084902
:1057A000C87FFEF73DFB064890F8200010B10120AD
:1057B000FFF720FD002102484175002016E7000098
:1057C000EC00002010B5C8234FF48062F74940F682
:1057D000F630FFF767FE10BD10B586B00446F4A0A2
:1057E00000680390F3A000680290F3A000680190A5
:1057F000F2A00068009004F0030003A9085C8DF893
:10580000140003A8C4F3C101405C8DF8150003A87F
:10581000C4F38111405C8DF8160004F0030002A966
:10582000085C8DF8100002A8C4F3C101405C8DF83B
:10583000110002A8C4F38111405C8DF8120005AA82
:10584000032140F22640FFF7B3FD18B14FF0FF30BF
:1058500006B010BD04AA032140F22A40FFF7A8FDBC
:1058600010B14FF0FF30F3E70198059000980490D5
:1058700004F0040058B19DF8140040F001008DF8C8
:1058800014009DF8100040F001008DF8100004F0A5
:10589000200058B19DF8150040F001008DF815006A
:1058A0009DF8110040F001008DF8110004F48070A3
:1058B00058B19DF8160040F001008DF816009DF8D3
:1058C000120040F001008DF8120005AA03214FF4E8
:1058D0008860FFF76DFD10B14FF0FF30B8E704AA04
:1058E000032140F23140FFF763FD10B14FF0FF306C
:1058F000AEE7B34804810020AAE71FB50446B048CC
:10590000007A00F0030054F820000190AC48007ABF
:1059100000F0040010B1019840420190A848007ABC
:10592000C0F3C10054F820000290A548007A00F0AE
:10593000200010B1029840420290A148007AC0F3C2
:10594000811054F8200003909D48008900F4807075
:1059500010B10398404203909A49019880FB0101DD
:10596000800F40EA810001909649029880FB011067
:10597000820042EA917002909249039880FB0110E4
:10598000820042EA917003900198000E8DF80000A9
:105990000198000C8DF801000198000A8DF80200B2
:1059A0000198C0B28DF803006A4604214FF4747068
:1059B000FFF7FEFC18B14FF0FF3004B010BD0298A5
:1059C000000E8DF800000298000C8DF8010002987E
:1059D000000A8DF802000298C0B28DF803006A46F2
:1059E00004214FF47570FFF7E3FC10B14FF0FF3066
:1059F000E3E70398000E8DF800000398000C8DF883
:105A000001000398000A8DF802000398C0B28DF8D7
:105A100003006A4604214FF47670FFF7C9FCCCE717
:105A200070B588B0064601A8FEF7BBFEBDF80400BD
:105A30000021C90341EA5045C4036148007A00F0DF
:105A4000030056F8200005905D48007A00F004003D
:105A500010B10598404205905948007AC0F3C10042
:105A600056F8200006905648007A00F0200010B149
:105A70000698404206905248007AC0F3811056F8CA
:105A8000200007904E48008900F4807010B10798FC
:105A9000404207900598C117A0FB042301FB043185
:105AA00000FB0510810041EA927005900698C1172D
:105AB000A0FB042301FB043100FB0510810041EA37
:105AC000927006900798C117A0FB042301FB0431D4
:105AD00000FB0510810041EA927007900598000EC6
:105AE0008DF808000598000C8DF809000598000A4B
:105AF0008DF80A000598C0B28DF80B000698000ECC
:105B00008DF80C000698000C8DF80D000698000A20
:105B10008DF80E000698C0B28DF80F000798000EA1
:105B20008DF810000798000C8DF811000798000AF6
:105B30008DF812000798C0B28DF8130002AA0C214C
:105B40004FF42570FFF734FC08B070BD30B585B058
:105B500004461DA207CA02AB07C3C82C03DD4FF0E1
:105B6000FF3005B030BDC82090FBF4F0401E85B278
:105B7000280A8DF80000E8B28DF801006A4602217B
:105B800040F21620FFF714FC10B14FF0FF30E8E7A9
:105B900002AA0C2140F6C120FFF70AFC10B14FF019
:105BA000FF30DEE7064884810020DAE7FC80000849
:105BB0004CCD6C000CC92C0036567600264666008B
:105BC000AC01002009E3CA02FEF2ABC4AAF1DFDF98
:105BD000BBAFDFDF0146FC488089088000207047AA
:105BE0002DE9FC4706460F4606F0070010B1B7F551
:105BF000C86F03DD4FF0FF30BDE8FC87384602F088
:105C000017F88146F14901F0C9FE80466846FEF763
:105C10004CFD9DF80000022806D0042816D0082864
:105C200026D0102848D135E04FF08D41404602F093
:105C300047F8814601F0C4FF84B2E549404602F0CE
:105C40003FF8814601F0BCFF85B238E04FF08C414F
:105C5000404602F035F8814601F0B2FF84B2DD49DA
:105C6000404602F02DF8814601F0AAFF85B226E0F9
:105C70004FF08B41404602F023F8814601F0A0FF2F
:105C800084B2D549404602F01BF8814601F098FFE6
:105C900085B214E04FF08A41404602F011F8814687
:105CA00001F08EFF84B2CD49404602F009F88146EA
:105CB00001F086FF85B202E04FF0FF309CE700BFA5
:105CC00020128DF80400E0B28DF8050028128DF83E
:105CD0000600E8B28DF8070006F00100A0B101AAA5
:105CE00002214FF4EA70FFF763FB10B14FF0FF3071
:105CF00082E70DF1060202214FF49270FFF758FB84
:105D000010B14FF0FF3077E706F00200A0B101AA12
:105D100002214FF4EC70FFF74BFB10B14FF0FF3056
:105D20006AE70DF1060202214FF49470FFF740FB81
:105D300010B14FF0FF305FE706F00400A0B101AAF8
:105D400002214FF4EE70FFF733FB10B14FF0FF303C
:105D500052E70DF1060202214FF49670FFF728FB7F
:105D600010B14FF0FF3047E7002045E738B5044653
:105D70000020009004F0010020B19DF8000040F0E8
:105D80003000009004F0020020B19DF8000040F0C7
:105D90000C00009004F0040020B19DF8000040F0D9
:105DA000030000906A4601214FF4A470FFF700FB46
:105DB00038BD38B50446012C01DA012402E0042C78
:105DC00000DD0424601EC0B200906A46012140F24A
:105DD0004F10FFF7EDFA38BD38B50446052094FBA7
:105DE000F0F085B228128DF80000E8B28DF80100BD
:105DF0006A4602214FF4EF70FFF7DAFA38BD38B582
:105E00000446052094FBF0F085B228128DF80000BE
:105E1000E8B28DF801006A4602214FF4ED70FFF7F9
:105E2000C7FA38BDF8B505460E464FF47A7095FBB3
:105E3000F0F000FB06F4200E8DF80000200C8DF829
:105E40000100200A8DF80200E0B28DF803006A46D6
:105E500004214FF4AE70FFF7ABFAF8BD38B5044635
:105E6000052094FBF0F084B220128DF80000E0B21F
:105E70008DF801006A4602214FF4AD70FFF798FAE1
:105E800038BD38B50446052094FBF0F084B22012EA
:105E90008DF80000E0B28DF801006A4602214FF44F
:105EA000AC70FFF785FA38BD38B5044614B94FF029
:105EB000FF3038BD6A4604214FF45870FFF7B5FA39
:105EC00010B14FF0FF30F4E79DF8000000069DF898
:105ED000011040EA01409DF8021040EA01209DF8BF
:105EE0000310084320600020E3E738B50446200E85
:105EF0008DF80000200C8DF80100200A8DF80200BA
:105F0000E0B28DF803006A4604214FF45870FFF7A1
:105F10004FFA38BD38B5044614B94FF0FF3038BDDC
:105F20006A4604214FF47170FFF77FFA10B14FF009
:105F3000FF30F4E79DF8000000069DF8011040EAEC
:105F400001409DF8021040EA01209DF8031008432B
:105F500000EB8000800020600020E0E738B50446B8
:105F60001420B4FBF0F4200E8DF80000200C8DF806
:105F70000100200A8DF80200E0B28DF803006A46A5
:105F800004214FF47170FFF713FA38BD38B5044699
:105F900064B120208DF8000028208DF80100302009
:105FA0008DF8020038208DF8030004E0A3220421BC
:105FB000684600F05FFC6A46042140F69E20FFF729
:105FC000F7F9FDF74FFE38BDAC0100200000484353
:105FD000000040460000C045000040450000C044AD
:105FE00038B5044664B1C0208DF80000C2208DF899
:105FF0000100C4208DF80200C6208DF8030004E0E3
:106000008B220421684600F035FC6A46042140F6E4
:106010009820FFF7CDF9FDF725FE38BD3EB50446C3
:106020006CB1FDA1D1E900208968CDE90020029181
:106030006A4609214FF49760FFF7BAF93EBDF9A20D
:10604000D2E900109268CDE9010200916A46092167
:106050004FF49760FFF7ACF9F0E73EB50446022035
:106060008DF80000CA208DF80100E3208DF80200B1
:1060700009208DF803006A4604216820FFF798F98B
:10608000A3208DF8000004F0400048B1C0208DF836
:106090000100C8208DF80200C2208DF8030006E040
:1060A000A3208DF801008DF802008DF8030004F4A0
:1060B000C07048B1C4208DF80400CC208DF80500D4
:1060C000C6208DF8060006E0A3208DF804008DF8A8
:1060D00005008DF80600A3208DF807008DF8080054
:1060E0008DF809006A460A2140F6A720FFF760F9FB
:1060F00004F0030018B120208DF8000002E0D82041
:106100008DF800006A46012140F6B620FFF750F9ED
:1061100004F0200018B10120FFF780FF02E000200A
:10612000FFF77CFF04F4C07008B304F4807060B122
:10613000B2208DF800008B208DF80100B6208DF87C
:1061400002009B208DF803000BE0B0208DF80000CA
:1061500080208DF80100B4208DF8020090208DF889
:1061600003006A46042140F6A220FFF721F904F05B
:10617000010020B3F8208DF800006A4601214FF499
:106180000B60FFF715F9FA210720FFF729FD07201B
:10619000FFF7ECFD0120FFF70CFE6420FFF71CFE6B
:1061A0004FF4FA70FFF72BFEC821A148FFF73AFE23
:1061B0002820FFF753FE0A20FFF763FE08E0D820EF
:1061C0008DF800006A4601214FF40B60FFF7F0F8EC
:1061D00004F0020018B1D9208DF8000002E0D820A8
:1061E0008DF800006A46012140F23D70FFF7E0F8AB
:1061F00004F0040018B10120FFF7F2FE02E00020D5
:10620000FFF7EEFE04F0100018B10120FFF7BEFE0C
:1062100002E00020FFF7BAFE44F0080085494881FB
:10622000FDF720FD00208349887304F0400018B179
:106230000846807B801D887304F4C07020B17D48BF
:10624000807B801D7B49887304F0140020B179485D
:10625000807B10307749887304F0030020B17548C3
:10626000807B001D7349887300203EBD0146714844
:1062700040890880002070472DE9F0410446E0780D
:1062800000F0C006E07800F03F05607800F0010003
:1062900098B1EF102846E91705EB5171C910A5EB2D
:1062A000C101491C01F0FF086248006820B1614843
:1062B000414602683846904700BF607800F0080009
:1062C00030B15C48406818B1B0115A4A51688847EB
:1062D0000020BDE8F08110B586B0044656A207CA7A
:1062E00003AB07C357A207CA8DE80700012C09D0EA
:1062F000022C0ED103AA0B2140F68220FFF758F89A
:1063000006B010BD6A460B2140F68220FFF750F818
:10631000F6E74FF0FF30F3E72DE9F04F8DB0074679
:10632000884615469946DDE9166B0024002030802A
:106330004049887B5A4605A9FEF78FFB18B1601EBD
:106340000DB0BDE8F08F3B48807A00F014000028C3
:1063500061D09DF8140000069DF8151040EA014038
:106360009DF8161040EA01209DF817100843286098
:106370009DF8180000069DF8191040EA01409DF8AC
:106380001A1040EA01209DF81B10084368609DF830
:106390001C0000069DF81D1040EA01409DF81E10EB
:1063A00040EA01209DF81F100843A8609DF82000D6
:1063B00000069DF8211040EA01409DF8221040EAB5
:1063C00001209DF823100843E86004F11000C4B2D6
:1063D000286800140190686800140290A8680014EE
:1063E0000390E8680014049001984043029901FB6F
:1063F0000100039901FB0100049901FB010ABAF1B4
:10640000706F02DBBAF1885F22DDFDF72BFC002004
:106410003080401E94E721E0B8AAB38DB4980D35C2
:106420005D000000B8AAAAAAB088C3C5C7000000D2
:1064300009E3CA02AC010020D8B1B9F38BA391B62D
:1064400009B4D900DAB1B9F38BA391B6DAB4DA00A2
:10645000B6F9000040F48070308000BF3448807A84
:1064600000F0400020B305A9601C085C095D40EA0B
:10647000012000B2A8F8000005A9E01C095C05AAEB
:10648000A01C105C41EA002000B2A8F8020005A997
:10649000601D095C201D105C41EA002000B2A8F8D4
:1064A0000400A01DC4B2B6F9000040F0080030801E
:1064B0001F48408900F4C07008B305A9601C085C3F
:1064C000095D40EA012000B2388005A9E01C095CA2
:1064D00005AAA01C105C41EA002000B2788005A942
:1064E000601D095C201D105C41EA002000B2B880EC
:1064F000A01DC4B2B6F9000040F0700030800C4816
:10650000807A00F0030018B105A90819FFF7B4FE5E
:106510004846FDF706FF002012E7014604480160E7
:10652000002070470146024841600020704700008B
:10653000AC010020FBF75EFC4FF41650FCF722FA8A
:106540004FA15448FCF7E8FAFCF708FCC820FBF719
:1065500085FD51A14F48FCF7DFFAD020FBF7B3FED1
:106560000446224650A14B48FCF7D6FAFDF788F8BE
:10657000FDF79AF8FBF73EFF6420FBF76FFD7EE026
:106580001420FBF76BFDFDF7FDF806214B48FCF7E7
:1065900057FB4A48C078B1280AD148480079B52845
:1065A00006D100204549C87006214448FCF73BFA53
:1065B0004248C078B3280AD140480079B72806D1AC
:1065C00000203E49C87006213C48FCF72CFA3B48A5
:1065D000C078B22809D139480079B62805D1FCF72E
:1065E000BDFB06213548FCF71EFA3448C078B428B4
:1065F00012D132480079B8280ED1FCF7BFFB4FF416
:10660000FA70FBF72BFDFCF7A9FB00202B49C870A3
:1066100006212A48FCF707FA2848C078B52809D18E
:1066200026480079B92805D1FCF7B8FB0621234894
:10663000FCF7F9F92148C078B62812D11F48007933
:10664000BA280ED1FCF7A2FB4FF4FA70FBF706FD57
:10665000FCF784FB00201949C87006211748FCF795
:10666000E2F91648C078B82809D114480079BC2846
:1066700005D1FCF77BFB06211048FCF7D4F97FE736
:10668000496E697420426C756520746F6F74682E52
:106690002E0D0A00004400404949432053746F7096
:1066A0002E2E0D0A0000000049494320496E6974EE
:1066B00020526573203D2025640D0A00BC01002096
:1066C000704700BFFEE700BFFEE700BFFEE700BF68
:1066D000FEE7704770477047704710B54C1084EA6A
:1066E000530404D54042C1F1000138BF491E1B428A
:1066F00004D55242C3F1000338BF5B1E00F0C6F858
:1067000014F0804F04D04042C1F1000138BF491E4F
:1067100014F0004F04D05242C3F1000338BF5B1E97
:1067200010BD00000FB4044910B503AA029800F090
:106730007DF910BC5DF814FB380000202DE9F04114
:106740000E460446002020622046E168884730B3A8
:10675000252805D0D4E901219047206A401CF2E7A2
:10676000E168204600278847050018D0A5F14100C0
:10677000192802D820354FF40067324629462046B2
:106780002760F9F70FFD40B1012804D0F61D26F06F
:1067900007060836D8E7361DD6E72846DAE7206A26
:1067A000BDE8F0812DE9F041064600241068752906
:1067B000314616A510D0AFF30080002802DA40421F
:1067C00013A507E031688A0701D512A502E0490741
:1067D00004D511A5012401E0AFF3008000210A22B5
:1067E00006F1240709E0B0FBF2FCB0FBF2F302FB78
:1067F0001C00303078541846491C0028F3D1234639
:106800002A463046BDE8F04100F0B7B8000000006D
:106810002D0000002B0000002000000040EA0103D2
:1068200010B59B070FD1042A0DD310C808C9121F39
:106830009C42F8D020BA19BA884201D9012010BD73
:106840004FF0FF3010BD1AB1D30703D0521C07E040
:10685000002010BD10F8013B11F8014B1B1B07D1A4
:1068600010F8013B11F8014B1B1B01D1921EF1D115
:10687000184610BD02F0FF0343EA032242EA024237
:1068800000F0E8B8704770477047704753EA020C51
:1068900000F069802DE9F04B4FF00006002B1FBF80
:1068A000B3FA83F503FA05F424FA05F65E4012BF45
:1068B0001643B2FA82F502FA05F4C5F120051EBFAF
:1068C00022FA05FC44EA0C04203556EA044C4FEA4F
:1068D000144418BF641C4FF000084FF000099042A8
:1068E00071EB030C39D3002919BFB1FA81F701FA12
:1068F00007F6B0FA80F700FA07F6C7F120071EBFC7
:1069000020FA07FC46EA0C062037B6FBF4FCA7EB9E
:106910000507103F07F01F0BCBF120060CFA0BFB0D
:106920002CFA06F644BFB3460026202FA4BF5E46CD
:106930004FF0000B5BEA060C08BF4FF0010B19EBA0
:106940000B09ABFB027C48EB0608C01B06FB02CC24
:106950000BFB03CC71EB0C01C1E70B460246414631
:106960004846BDE8F08B13B54FF000004FF0000132
:10697000AFF30080BDE81C4070472DE9F0470D469D
:1069800099469246044600F124080168880604D519
:10699000E06921F01001216000E00120A84201DD42
:1069A000471B00E00027A1697A1902EB0900081AC9
:1069B000A0612078C00602D42046AFF300800026F4
:1069C00008E0D4E901211AF806009047206A401C2B
:1069D000761C20624E45F4DB2078C0060AD520469E
:1069E000AFF3008006E0D4E9012130209047206A0F
:1069F000401C2062381EA7F10107F4DC07E0D4E94F
:106A0000012118F805009047206A401C2062281ECA
:106A1000A5F10105F3DC2046AFF3008020780006E5
:106A200002D50220BDE8F0870120FBE7074B70B5D7
:106A30000D467B4400F033F80446284600F042F847
:106A400010B14FF0FF3070BD204670BD0BB5FFFF99
:106A50004FF000020429C0F0128010F0030C00F087
:106A60003780CCF1040CBCF1020F18BF00F8012BE9
:106A7000A8BF20F8022BA1EB0C0100F029B85FEAB7
:106A8000C17C24BF00F8012B00F8012B48BF00F89F
:106A9000012B704701694A1C02610878704700B5F4
:106AA0008FB0CDE901310021059105497944CDE947
:106AB000031011466846FFF741FE0FB000BD00000D
:106AC000E5FFFFFF007B00F0800070474FF0000201
:106AD00000B5134694469646203922BFA0E80C50D4
:106AE000A0E80C50B1F12001BFF4F7AF090728BFAF
:106AF000A0E80C5048BF0CC05DF804EB890028BF2B
:106B000040F8042B08BF704748BF20F8022B11F053
:106B1000804F18BF00F8012B7047000000487047F5
:106B2000FC0100207546FFF7F9FFAE4605006946F7
:106B3000534620F00700854618B020B5F9F758FBFA
:106B4000BDE820404FF000064FF000074FF000086E
:106B50004FF0000B21F00701AC46ACE8C009ACE8EF
:106B6000C009ACE8C009ACE8C0098D46704710B553
:106B70000446AFF300802046BDE81040F9F724BB7F
:106B8000490050EAC12018BF04204A0D18BF40F048
:106B9000010040F2FF72B2EB515F08BF40F002000B
:106BA000012808BF052070472DE9F0414F1E00EB7A
:106BB000C7010446D1E9000115461E4637F006021A
:106BC0000DD02A46334600F05BFC7F1E04EBC70362
:106BD000D3E9002300F04CFA37F00602F1D1022F7E
:106BE00025D0042F13D0062F18BFBDE8F0812A4608
:106BF000334600F045FCD4E90A2300F039FA2A466E
:106C0000334600F03DFCD4E9082300F031FA2A466F
:106C1000334600F035FCD4E9062300F029FA2A4671
:106C2000334600F02DFCD4E9042300F021FA2A4673
:106C3000334600F025FCD4E9022300F019FA2A4675
:106C4000334600F01DFCD4E90023BDE8F04100F01C
:106C50000FBA012201F0E3B900F00ABA024A00209B
:106C6000110701F0DCB9000001FDFFFF2DE9F84F2D
:106C700004460D4621F0004000917349814211DC29
:106C80007249884201DC06D12CB120462946BDE874
:106C9000F84FFFF7DEBF6E48002DCCBF6D496E493F
:106CA000BDE8F88F6D49814211DD6D498142D8BF41
:106CB0004FF0FF366DDD20462946FFF761FF0428BF
:106CC00008BFFFF7CBFF20462946BDE8F88F65498E
:106CD000654F25F00045814233DD6449814219DD6D
:106CE000002632464FF080432046294600F0C0F986
:106CF00080468A4601222046294601F090F900226A
:106D00003B4600F0C7FC4246534600F061FA044699
:106D10000D463EE001260022BA463B462046294663
:106D200000F0A6F980460F46002253462046294629
:106D300000F0B0FC42463B4600F04AFA04460D46DD
:106D400027E04B4981421BDDDFF828A10226002203
:106D500053462046294600F093FB00223B4600F0B4
:106D600087F980460F46002253462046294600F008
:106D700091FC42463B4600F02BFA04460D4608E0E3
:106D8000032622462B4600203B4900F021FA044608
:106D90000D4622462B461046194600F071FB8B46E5
:106DA000824602460B4600F06BFB0746024633481C
:106DB00088460B4606217844FFF7F6FE52465B46AE
:106DC00000F05EFB82462E488B463A46434605213C
:106DD0007844FFF7E9FE3A46434600F051FB02468D
:106DE0000B46002E504659460CDA00F041F9224677
:106DF0002B4600F045FB01B022462B46BDE8F04F84
:106E000000F03CBC00F034F922462B4600F038FB81
:106E10001C4A7A4402EBC603D3E9002300F03AFC93
:106E200022462B4600F036FC174A7A4402EBC60392
:106E3000D3E9002300F022FC009A002AB8BF81F0B9
:106E40000041BDE8F88F0000000010440000F07F12
:106E5000182D4454FB21F93FFB21F9BF0000DC3F12
:106E60000000203E0000F33F0000F03F0000E63F3E
:106E7000008003400000F83F0000F0BFA61F0000A4
:106E8000641F0000021F0000CA1E00002DE9F04D23
:106E90009446CCF1000423F000464CEA0404524F1F
:106EA00046EAD4749A46884621F00042BC4206D88D
:106EB000454240EA050442EAD474BC4204D9BDE824
:106EC000F04D6246FFF7C8BEAAF14055A5F17F65B7
:106ED00055EA0C040BD0022404EAAA74434DDFF8EF
:106EE00010E144EAD87452EA000B04D00CE0BDE88B
:106EF000F04DFFF7BBBE002C14BF012CBDE8F08D98
:106F0000022C30D0032C32D056EA0C0B0AD0BE42F1
:106F100020D1BA4209D126F0804622F08042334681
:106F2000114617E000291ADB25E0DFF8C8B0FB4462
:106F3000002C04BFDBE90001BDE8F08D012C02BF8D
:106F4000DBE9000181F00041BDE8F08D022C0AD0A0
:106F5000032C0CD0BA4212D1B8F1000F0BDA23483F
:106F60002549BDE8F08D28462449BDE8F08D284626
:106F70007146BDE8F08D1D482149BDE8F08D921B9A
:106F800012153C2AC4BF19481D490EDCBAF1000F86
:106F9000BEBF12F13C0F0020014606DB624600F046
:106FA00017F921F00041FFF761FE002C08BFBDE892
:106FB000F08D012C04BF81F00041BDE8F08D114A35
:106FC000114B022C07D000F065FB2A46BDE8F04DBE
:106FD0000A4B00F05FBB00F05DFB2A46BDE8F04DB8
:106FE000064B00F04BBB00000000F07F182D44540E
:106FF000FB2109C05E1E0000FB21F9BFFB210940F7
:10700000FB21F93F075C143326A6A13C21F0004286
:10701000A2F16052B2F5801F01F0004328BFD2F107
:107020007F6C0BD95FEA001C43EAC20242EB50704E
:1070300018BF704728BF20F001007047B2F5801FCD
:10704000BCBF184670474FEA410C1CF5001F02D226
:10705000084600F0FCBE70B500F0BCFA00000089E4
:10706000FFF7F6BF4FF00040A0F58000704700002A
:1070700010B591EA030F48BF83F0004300F112837B
:10708000841A71EB030C05D2121943EB0C03001B9D
:1070900061EB0C01DFF824E14FEA1154A4EB135C1F
:1070A0001EEA430F18BF9EEA445F73D023EA0E0323
:1070B000DCF1200E21EA045143F4801332D322FA8A
:1070C0000CFE10EB0E0023FA0CFE41EB0E01CCF18E
:1070D000200E03FA0EFE10EB0E0051F10001B1F587
:1070E000801FCCF1200E32D201EB045112FA0EF2C5
:1070F000BDE8104058BF7047401C38BF5FEA4202ED
:1071000018BF7047002814BF20F0010041F10001B2
:107110004FEA410313F5001F38BF7047A1F1C0418A
:1071200000F0A6BA012A43EB0302ACF1200CDCF11B
:107130001F0E32BF4FF0000E23FA0CF310EB0300CA
:1071400041EB0451B4EB115FD0D0A1EB045101F538
:10715000801149085FEA300001EB04510ED350F171
:10716000000038BF12FA0EFE08D1BDE81040C9E792
:10717000401C38BF5FEA4202CAD1C3E7BDE81040F5
:107180004FEA410313F5001F38BF7047A1F1C0411A
:1071900000F06EBA9EEA445F08D011EA5E0FBDE8C7
:1071A000104004BF01F0004100207047BDE81040CE
:1071B00070B500F00FFA00BF64FBBE3E0000E0FFB8
:1071C00002494FF0000000F0F8BE00BF0000F87F59
:1071D0002DE9C04130B4DFF8A0C23CEA111418BF59
:1071E0003CEA131400F0EC8081EA03051CEA111458
:1071F00044EAD57418BF1CEA131500F0C780A4EB4D
:1072000005044FF0004545EAC12145EAC32341EAA0
:10721000505143EA525304F17F74994204F500340B
:107220004FEAC0204FEAC22208BF904200F09C8083
:107230004FEA13650FF24016765D4FEA134506FBE1
:1072400005F7C7F1807706FB07F74FEAD737A7FBAB
:1072500003687642C8F58038A7FB06CE38BFA8F190
:10726000010807FB08E64FF0000EA6FB028CE6FBC8
:1072700003CEDCF1000CCEF1004E38BFAEF1010EB2
:10728000A6FB0C584FF000074FF00005E6FB0E87F9
:10729000A1FB08C6A0FB07CE16EB0E0645F10005C4
:1072A000E1FB076515F1E04E7EBFA4F580345FEA8F
:1072B00046066D4116F1800745F100054FEA172794
:1072C0004FEA066647EA0567A6F1DE46B6F1805F3B
:1072D0004FEA15251FD9384624F0010C05EBC4717F
:1072E000BCF1FE6F01EB0C1102D8F0BCBDE80081CF
:1072F00024425CBF01F5801E9EEAC47F02D4F0BC2C
:10730000BDE80081244238D4F0BCA1F1C041BDE801
:10731000004100F0ADB94FEAD22242EA43524FEAAF
:10732000D323A7FB02864FEAD02040EA415007FB57
:1073300003661EEA0E0F4FEAD12105FB026658BF15
:10734000A6EB0056B6EB00564FEA520E4EEAC37E4D
:1073500018EB0E0E56EB530EBDD518EB02085E412E
:107360007F1C55F10005B6E74FF480154FF000077C
:107370004FF000064FF00008ADE7F0BC4FF0000002
:1073800001F1C04101F00041BDE8008111EA0C1F8C
:107390000CEA131500D00CE013EA0C1F00F0258056
:1073A0004FF00000F0BC81EA030101F00041BDE8AC
:1073B0000081F0BCBDE8004181EA030100F058B94A
:1073C000F0BCBDE8004170B500F004F9097EFC3E58
:1073D00000F007B881EA03014FF0000001F000411E
:1073E000704781EA030100F043B9F0BCBDE80041F9
:1073F0004FF0000021497047FFFDFBF9F7F5F4F26B
:10740000F0EEEDEBE9E8E6E4E3E1E0DEDDDBDAD83F
:10741000D7D5D4D3D1D0CFCDCCCBCAC8C7C6C5C49D
:10742000C2C1C0BFBEBDBCBBBAB9B8B7B6B5B4B3B4
:10743000B2B1B0AFAEADACABAAA9A8A8A7A6A5A49F
:10744000A3A3A2A1A09F9F9E9D9C9C9B9A99999863
:107450009797969595949393929191908F8F8E8E06
:107460008D8C8C8B8B8A8989888887878685858493
:1074700084838382828181800000FF070000F87F7F
:10748000DFF848C170B51CEA111E1EBF1CEA1315B7
:107490009EEA0C0F95EA0C0F00F06F8081EA03045E
:1074A00023EA4C134EEAD47E21EA4C1141F48011B8
:1074B00043F48013AE44A1FB024CA0FB0365AEF184
:1074C0007F7E361955EB0C05A1FB034C4CF10003F4
:1074D000A0FB021C16EB0C06654153F100030942A8
:1074E00018BF46F0010613F4007F0BD14FEA0331B9
:1074F0004FEA0530340341EA155140EA16506FF067
:1075000003020AE04FEAC3214FEAC520F40241EA30
:10751000555140EA56506FF0020202EB2E4201EB49
:10752000025585EACE710AD05FEA440C18BF24F0F8
:10753000004450F1000041F1000120EAD47040F213
:10754000FE7C624500D270BDA84214BF4FF080445B
:107550004FF04044002E08BF0024BEF1806FA8BF4A
:10756000A1F1C041BDE8704080F282804FF0000080
:1075700001F1C04101F0004170479EEA0C0F0CEA96
:10758000131518BF95EA0C0F06D04FF0000081EAE2
:10759000030E0EF0004170BD00F01CF88900013EA2
:1075A00000F007B800F009B84FEA430C5FEA5C5CF2
:1075B00008D081EA030100F05BB84FEA410C5FEAB2
:1075C0005C5CF6D14FF00000014970470000FF07F6
:1075D0000000F87F0EF1020E2EF0030E5EF8046B31
:1075E000364205D4012A43EB030515F5001F12D8D6
:1075F000012841EB010C1CF5001F0CD80ED14FEAFD
:10760000D17C15F5001F0CEB4C0C0CF1020C08BFE3
:107610004CEBD37C04E04FF0080C01E04FEAD37C44
:107620000CEB4C0526FA05F606F00706B6F1040C3D
:1076300006D20EEB860CBDE870404CF0010C6047A2
:10764000DFE80CF0090B02024FF000414FF00000A0
:10765000A1F5002170BD19461046012851EB010427
:1076600018BFD4F5001484BF002001F0004170BDA4
:107670000808A0F500114FEA3101704791EA030FA5
:1076800010B581F000413FF5FBAC83F0004300F002
:1076900009B8000010B591EA030F48BF83F000431A
:1076A0003FF5EEAC841A71EB030C07D212198CF083
:1076B000004C43EB0C03001B61EB0C01DFF8A4E171
:1076C0004FEA1154A4EB135C1EEA430F18BF9EEA65
:1076D000445F00F0B08023EA6E03524221EA045175
:1076E000C3EB6E0338BF5B1EDCF1200E25D322FAFC
:1076F0000CFE10EB0E0043FA0CFE41EB0E01CCF138
:10770000200E03FA0EFE10EB0E0051F10001CCF139
:10771000200E29D412FA0EF201EB0451BDE81040FC
:1077200058BF7047401C1CBFB2F1004F7047002883
:107730000CBF491C20F00100704712EB020E43EB16
:10774000030218BF4FF0010E4EEA4202ACF1200CCA
:10775000DCF11E0E54D943FA0CFE10EB0E0051F171
:10776000FF31CCF11E0ED5D50EF1010E12FA0EFE30
:10777000404141EB010101EB445C5FEA5C5C10D9E4
:1077800010EBDE7001EB045138BFBEF1004FBDE8D5
:10779000104018BF704700280CBF491C20F00100A2
:1077A000704730D24FEAD42C11F5001124F4006454
:1077B0001BD0B1FA81F20B3AA41AA41ED2F1200315
:1077C000914030FA03F31943904001EBCC71002C47
:1077D00001EB0451BDE81040A8BF704701F1C04162
:1077E0004FF0000001F000417047B0FA80F310FA4A
:1077F00003F100D110BDE41A173C4805C90AE4E7BB
:1078000001EB045110BD491001EB0451BDE81040DB
:107810004FEA300002E04FF0000170474A0008BF15
:107820000042F8D0B2F5001F28BF704701F00041B8
:107830004FF0000070479EEA445F07D011EA5E0FE8
:10784000BDE8104004BF002100207047BDE8104093
:1078500070B5FFF7BFFE00BF40DFF63E83F000418A
:10786000104670470000E0FF43004FEAD30C4FEA98
:107870003C0C43401FBF40070CF1605113F0FE4F1A
:1078800070471CF0006F03D100200CF000417047DE
:107890000CF0004343EA507010B540EACC0000F011
:1078A00090FA00BF000000924FEA0001FFF7E0BE2F
:1078B0004FF000414FF00000A1F50021704700009B
:1078C00090EA010F48BF81F0004100F10883421A9D
:1078D0003CBF801A89184FEAD0524FF07F4C1CEA07
:1078E000410FA2EBD15318BF9CEA026F00F03B801E
:1078F0004FF0004C4CEA00204CEA012121FA03FC35
:1079000010EB0C0C1ED202F1FF325FEA1C2040EBA0
:10791000C25038BF70471CF07F0F4FEA400C18BFB1
:10792000BCF17F4F38BF7047C3F12003994008BFB7
:1079300020F00100BCF17F4F38BF7047A0F1C0407C
:1079400000F085BA4FEA3C00000A40EBC25028BF65
:107950001CF0FF0F4FEA400CE6D018BFBCF17F4F80
:1079600038BF7047EAE79CEA026F05D010EA5C0F67
:1079700008BF00F00040704710B500F022FA00BFC9
:1079800064FBBE3E401058BFC0F14040491058BF94
:10799000C1F140418142EFF3008070474FF47F0C0A
:1079A0001CEAD0121EBF1CEAD11392EA0C0F93EA14
:1079B0000C0F00F0858090EA010F48BF42F48072FE
:1079C00040F4000C41F400002CF07F4120F07F4097
:1079D00000B58142A2EB03020FF2081CACEB504E43
:1079E000C0F100009EF800E04FEA4E0E00FB0EFCD6
:1079F00038BF49004FEA2C1C02F5FA020CFB0EF3CB
:107A00004FEACE1E4FEA112C4FEAC1210EEB635E06
:107A100042EB22420EFB0CFC4FEA1C5300FB03110D
:107A20004FEA112C4FEA01310EFB0CFC4FEADC4C03
:107A300000FB0C11C14228BF09184CEB03335DF861
:107A400004EB10EB410143EBC250B2F57C0F38BFA1
:107A5000704729D512F0F00F1CBF00F1C04000F0B4
:107A600000407047008182838485868788898B8C5B
:107A70008D8E8F919293959697999A9C9D9FA0A297
:107A8000A3A5A7A8AAACAEB0B2B3B5B7B9BCBEC0E7
:107A9000C2C5C7C9CCCED1D4D7D9DCDFE2E6E9EC88
:107AA000F0F3F7FAFE0000004FEA400C0CF1807C86
:107AB000BCF17E4F28BF7047B0F1C04000F0C7B99D
:107AC00090EA010F0CEAD11348BF42F4807262457C
:107AD00038BF634507D213F47F0F16D080EA010048
:107AE00000F00040704710B500F06BF9097EFC3ED5
:107AF00000F005B880EA010000F00040704780EA1D
:107B0000010000F0004000F0A2B912F47F0F04BFA2
:107B10000248704780EA010000F099B90000C07F78
:107B200050EA010C00F113801CF5000F58BFBCF5A2
:107B3000000F01D48842704707D710F5000F58BFD7
:107B400011F5000F15D488427047894270471CF523
:107B5000000F04D5BCF5000FF7D5814270474FF0F8
:107B6000807C1CEB400F38BF1CEB410F01D28142DF
:107B7000704710B500F025F9922449004FF00050ED
:107B80004FF08051FFF7FEBE41000B0ED3F19E0275
:107B900008D950F400034FEA032323FA02F048BF48
:107BA0004042704710B500F00CF900BF49922480A4
:107BB000002070476FF0004282EA2000704700000A
:107BC000C10DD1F19E0206DB4FEA002343F00043D2
:107BD00023FA02F07047004207D54FEA4001B1F1A5
:107BE000FE4F02D24FF00000704710B500F0E9F8E8
:107BF00049922480002070476FEA200070470000FF
:107C000010F0004148BF4042B0FA80F310FA03F28E
:107C1000C3F19D030BD051EAC35101EB122053066F
:107C200038BF704700F1010008BF20F00100704725
:107C3000B0FA80F310FA03F2C3F19D030AD0D9051C
:107C400001EB1220530638BF704700F1010008BF56
:107C500020F001007047000050EA010C00F1138091
:107C60001CF5000F58BFBCF5000F01D488427047C7
:107C700007D710F5000F58BF11F5000F15D4884233
:107C80007047894270471CF5000F04D5BCF5000F02
:107C9000F7D5814270474FF0807C1CEB400F38BF16
:107CA0001CEB410F01D28142704710B500F089F8FA
:107CB000922449004FF000504FF08051FFF762BE10
:107CC0004FF47F0C1CEAD0121EBF1CEAD11392EABB
:107CD0000C0F93EA0C0F00F0478090EA010F48BFA9
:107CE00042F480724FF0004C4CEA00204CEA012133
:107CF00002EB0302A0FB0113A2F50002002918BF4A
:107D000043F001035B0028BF4FEA330342EB2242FA
:107D10005FEA132C4CEBC2502EBFBCEB436FB2F5A5
:107D20007C0F70474FEA036CBCF1004F08BF20F096
:107D30000100B2F57C0F38BF70470BD582F0FF020F
:107D400012F5803FC8BF704700F1C040D8BF00F0B7
:107D50000040704700F5000C5FEA4C0C48BF7047CC
:107D6000B0F1C04000F073B890EA010F0CEAD113F3
:107D700048BF42F48072624538BF634504D280EA4E
:107D8000010000F00040704710B500F01AF800BF85
:107D90008900013E00F007B800F009B85FEA410C25
:107DA0005FEA1C6C08D080EA010000F050B85FEA7E
:107DB000400C5FEA1C6CF6D14FF00040A0F580004B
:107DC00070470EF1020E2EF0030E5EF8044B2442B3
:107DD00004D44FEA4102B2F17F4F11D84FEA400379
:107DE000B3F17F4F0CD80ED14FEAD07CB2F17F4F68
:107DF0000CEB4C0C0CF1020C08BF4CEBD17C04E0FA
:107E00004FF0080C01E04FEAD17C0CEB4C0324FA54
:107E100003F404F00704B4F1040C06D20EEB840C56
:107E2000BDE810404CF0010C6047DFE80CF007089B
:107E300002024FF00040A0F5800010BD084642004D
:107E400018BFD2F1807288BF00F0004010BDFF2142
:107E500041EAD050C005704751EA000C00F1138090
:107E60001CF5000F58BFBCF5000F01D481427047CC
:107E700007D711F5000F58BF10F5000F15D4814238
:107E80007047894270471CF5000F04D5BCF5000F00
:107E9000F7D5884270474FF0807C1CEB410F38BF0C
:107EA0001CEB400F01D28842704780EA010081EA52
:107EB000000180EA0100FFF7F8BE80F0004090EA80
:107EC000010F7FF504AD81F0004100F008B800001B
:107ED00090EA010F48BF81F000413FF5F8AC421A2B
:107EE00004D882F00042A0EB020011444FEAD052C5
:107EF0004FF07F4C1CEA410FA2EBD15318BF9CEA14
:107F0000026F4AD04FF0004C4CEA00204CEA0121AD
:107F100021FA03FCB0EB0C0C0FD412F0FE0F36D09C
:107F20005FEA4C001DD5001240EBC25038BF7047CD
:107F30001CF03F0F18BF70470BE0A2F101025FEA8F
:107F40001C2040EBC25038BF70471CF07F0F18BF99
:107F50007047C3F12003994014BF401E20F0010078
:107F6000704780084FEA122308BF7047B0FA80FCC0
:107F7000A2EB0C02CCF1280C60FA0CF093EA122F61
:107F800004BF00EBC25070474FEAC3707047130A3A
:107F90005FEADC1008BF7047F6E79CEA026F04D086
:107FA00010EA5C0F08BF0020704710B5FFF709FF0B
:107FB00040DFF63E81F0004070470CF00F03092BC4
:107FC00008BF082000F059800A2B0BD0082B18BFDF
:107FD000704708BF1CF0400F0AD04FF000004FF070
:107FE000000170471CF0400F18BF4FF00040704771
:107FF0001CF0100F08D020F0704300F07F4242EADE
:10800000D3014FEA4370704700F0604021F07F4297
:1080100042EA000201F07F4040EA727070474FF080
:10802000FF0C4CF4E06C1CEA11531CBF9CEA030CDF
:108030009445C2BFDA4201EB02517047002B0DD0CC
:10804000BCF1000F0FD0002A01F00041A4BF41F0A5
:10805000E04141F07F614FF00000704701F00041C6
:108060004FF00000704750EA01334FF09B0C18BFEF
:108070004CF0806C7FF4A4A870471CF4801F11D0D2
:108080001CF4E02F03D06FEACC31490070474FF069
:108090004050EFF3008222F0704242EA000282F385
:1080A000008870474FF0000070470000680000042F
:1080B00076005401F7FD000175191A0C6A231B1C88
:1080C0001F207274433B4138393A6B6C376F06247A
:1080D0006D6E7000830000000008000000010018B1
:1080E00032000500000020410000D242295C0F3E12
:1080F0009A99993E3333733F295C0F3E000070001C
:10810000000000240000000200030000006500548D
:10811000FFEF0000FA80000B12820001030C30C355
:108120000E8C8CE914D5400213710F8E3883F883BE
:108130003000F883258EF8833000F883FFFFFFFFBF
:108140000FFEA9D6240004001A8279A10000003C89
:10815000FFFF00000010000038836FA2003E0330D4
:108160004000000002CAE3093E8000002000000039
:10817000000000004000000060000000000C000053
:10818000000C186E000006920A16C0DFFFFF0256B0
:10819000FD8CD377FFE1C496E0C5BEAA00000000C5
:1081A000FFFF0B2B00001657000003594000000092
:1081B00000001DFA00026C1D000000003FFFDFEB15
:1081C000003EB3B6000D227800002F3C00000000F6
:1081D000001942B5000039A20000B365D90E9FC94D
:1081E0001DCF4C3430000000500000003BB67AE850
:1081F0000064000000C80000000000001000000043
:108200001000FA921000225E000D229F0001000073
:1082100000320000FF46000063D4000010000000A0
:1082200004D6000004CC000004CC00000000107252
:1082300000000040000000000000000000060002F6
:1082400000050007000000000064000000000000BE
:108250000000000500050064002000000000000090
:108260000000000000004000000003000000003299
:10827000F8980000FF650000830F0000FF9BFC00E2
:1082800000000000000000000000000000000000EE
:1082900000000000000000000000000000000000DE
:1082A000000000000000000000001000400000007E
:1082B000000000060000B26A000200000001FB831B
:1082C0000068000000D9FC007CF1FF830000000082
:1082D00000650000006403E8006400280000002539
:1082E0000000000016A000000000100000001000B8
:1082F000002F0000000001F4000010000028000022
:10830000FFFF4581FFFFFA7200000000000000003F
:10831000004400050005BAC6004778A2000000012D
:108320000000000000000600000000140000254DC1
:10833000002F706D000005AE000C02D000000000A0
:10834000000000000000000000000000001B000012
:1083500000000000000000000000000000640000B9
:108360000008000000000000000000000000000005
:1083700000000000000000000000000000000000FD
:1083800000000000000000000000000000000000ED
:1083900000000000000000000000000000000000DD
:1083A00000000000000000000000000000000000CD
:1083B000000000000000000000000000001B0000A2
:1083C0000000000000000000000E000E00000AC7C0
:1083D0000004000000000032FFFFFF9C00000B2B98
:1083E000000000020000000100000064FFE5000042
:1083F000000000000000000000000000000000017C
:1084000000000000000100000000000000018000EA
:108410000001800000018000002426D3000000003D
:1084200000000000000600100096003C0000000064
:108430000000000000000000000000000C0A4E6870
:10844000CDCF770950166759C619CE8200000000BB
:10845000000000000000000000000000000000001C
:108460000000000017D78400030000000000000097
:1084700000000000C7938F9D1E1B1C190000000008
:1084800000000000000000000000000000000000EC
:1084900000000000020318850000400000000003F7
:1084A0000000000300000000000000004000000089
:1084B00000000000000000000000000000000000BC
:1084C00000000000000000000000000000000000AC
:1084D000000000000000000000000000000000009C
:1084E000677DDF7E72902E554CF6E6880000000016
:1084F000000000000000000000000000D8DCB4B85C
:10850000B0D8B9ABF3F8FAB3B7BB8E9EAEF132F583
:108510001BF1B4B8B08097F1A9DFDFDFAADFDFDF9E
:10852000F2AAC5CDC7A90CC92C97F1A98926466620
:10853000B28999A92D557DB0B08AA896365676F1A4
:10854000BAA3B4B280C0B8A89711B28398BAA3F006
:10855000240844106418B2B9B49883F1A329557D56
:10856000BAB5B1A38393F0002850F5B2B6AA8393AD
:1085700028547CF1B9A3829361BAA2DADEDFDB81F1
:108580009AB9AEF5606870F1DABAA2DFD9BAA2FA88
:10859000B9A38292DB31BAA2D9BAA2F8DF85A4D0FE
:1085A000C1BBAD83C2C5C7B8A2DFDFDFBAA0DFDFC2
:1085B000DFD8D8F1B8AAB38DB4980D355DB2B6BA8C
:1085C000AF8C96198F9FA70E161EB49AB8AA872C47
:1085D000547CBAA4B08AB691325676B28494A4C8B8
:1085E00008CDD8B8B4B0F19982A82D557D98A80EC1
:1085F000161EA22C547C92A4F02C5078F184A898DA
:10860000C4CDFCD80DDBA8FC2DF3D9BAA6F8DABA94
:10861000A6DED8BAB2B68696A6D0F3C841DAA6C806
:10862000F8D8B0B4B882A892F52C548898F135D90E
:10863000F418D8F1A2D0F8F9A884D9C7DFF8F883E4
:10864000C5DADF69DF83C1D8F40114F1A8824EA82E
:1086500084F311D182F5D992289788F109F41C1C72
:10866000D884A8F3C0F9D1D99782F129F40DD8F3B1
:10867000F9F9D1D982F4C203D8DEDF1AD8F1A2FA0F
:10868000F9A88498D9C7DFF8F8F883C7DADF69DF7B
:10869000F883C3D8F40114F198A8822EA884F311AA
:1086A000D182F5D992509788F109F41CD884A8F3A7
:1086B000C0F8F9D1D99782F149F40DD8F3F9F9D17D
:1086C000D982F4C403D8DEDFD8F1AD8898CCA809EC
:1086D000F9D98292A8F57CF1883ACF944A6E98DB5A
:1086E0006931DAADF2DEF9D88795A8F221D1DAA5A1
:1086F000F9F417D9F1AE8ED0C0C3AE82C684C3A838
:108700008595C8A588F2C0F1F4010EF18E9EA8C629
:108710003E56F554F18872F40115F19845856EF5D1
:108720008E9E0488F142985A8E9E068869F4011C38
:10873000F1981E1108D0F504F11E97020298362513
:10874000DBF9D985A5F3C1DA85A5F3DFD88595A82E
:10875000F309DAA5FAD88292A8F578F1881A849FED
:1087600026889821DAF41DF3D8879F39D1AFD9DF55
:10877000DFFBF9F40CF3D8FAD0F8DAF9F9D0DFD945
:10878000F9D8F40BD8F3879F39D1AFD9DFDFF41DC7
:10879000F3D8FAFCA869F9F9AFD0DADEFAD9F88F84
:1087A0009FA8F1CCF398DB45D9AFDFD0F8D8F18F93
:1087B0009FA8CAF38809DAAF8FCBF8D8F2AD978DAE
:1087C0000CD9A5DFF9BAA6F3FAF412F2D8950DD1B7
:1087D000D9BAA6F3FADAA5F2C1BAA6F3DFD8F1BA8C
:1087E000B2B68696A6D0CAF349DAA6CBF8D8B0B40A
:1087F000B8D8AD84F2C0DFF18FCBC3A8B2B68696ED
:10880000C8C1CBC3F3B0B48898A821DB718D9D712A
:10881000859521D9ADF2FAD88597A828D9F408D83A
:10882000F28D29DAF405D9F285A4C2F2D8A88D9484
:1088300001D1D9F411F2D88721D8F40AD8F284985A
:10884000A8C801D1D9F411D8F3A4C8BBAFD0F2DEC7
:10885000F8F8F8F8F8F8F8F8D8F1B8F6B5B9B08A39
:1088600095A3DE3CA3D9F8D85CA3D9F8D87CA3D9CA
:10887000F8D8F8F9D1A5D9DFDAFAD8B18530F7D927
:10888000DED8F830ADDADED8F2B48C99A32D557D60
:10889000A083DFDFDFB591A0F629D9FBD8A0FC29A2
:1088A000D9FAD8A0D051D9F8D8FC51D9F9D879D96A
:1088B000FBD8A0D0FC79D9FAD8A1F9F9F9F9F9A037
:1088C000DADFDFDFD8A1F8F8F8F8F8ACDEF8ADDED3
:1088D0008393AC2C547CF1A8DFDFDFF69D2CDAA06B
:1088E000DFD9FADB2DF8D8A850DAA0D0DED9D0F83D
:1088F000F8F8DB55F8D8A878DAA0D0DFD9D0FAF8A4
:10890000F8F8F8DB7DF8D89CA88CF530DB38D9D0A6
:10891000DEDFA0D0DEDFD8A848DB58D9DFD0DEA06C
:10892000DFD0DED8A868DB70D9DFDFA0DFDFD8F1C9
:10893000A888902C547C98A8D05C38D1DAF2AE8C00
:10894000DFF9D8B087A8C1C1B188A8C6F9F9DA366D
:10895000D8A8F9DA36D8A8F9DA36D8A8F9DA36D8A4
:10896000A8F9DA36D8F78D9DADF818DAF2AEDFD86F
:10897000F7ADFA30D9A4DEF9D8F2AEDEFAF983A762
:10898000D9C3C5C7F1889BA77AADF7DEDFA4F88409
:108990009408A797F300AEF29819A488C6A3948808
:1089A000F632DFF28393DB09D9F2AADFD8D8AEF82A
:1089B000F9D1DAF3A4DEA7F1889B7AD8F38494AED8
:1089C00019F9DAAAF1DFD8A881C0C3C5C7A3928379
:1089D000F628ADDED9F8D8A350ADD9F8D8A378AD34
:1089E000D9F8D8F8F9D1A1DADEC3C5C7D8A18194E6
:1089F000F818F2B089ACC3C5C7F1D8B8B4B097863F
:108A0000A8319B069907AB9728889BF00C2014404F
:108A1000B0B4B8F0A88A9A285078B79BA8295179A1
:108A2000247059446938644831F1BBAB88002C5438
:108A30007CF0B38BB8A804285078F1B088B497269E
:108A4000A85998BBABB38B02264666B0B8F08A9C97
:108A5000A82951798B2951798A2470598B20587112
:108A60008A4469388B3940688A6448318B30496060
:108A700088F1AC002C547CF08CA804285078F18844
:108A80009726A85998AC8C02264666F0899CA8299E
:108A90005179247059446938644831A988092059AA
:108AA00070AB11384069A8193148608CA83C415C12
:108AB000207C00F187981986A86E767EA999882D6A
:108AC000557DD8B1B5B9A3DFDFDFAED0DFAAD0DEE8
:108AD000F2ABF8F9D9B087C4AAF1DFDFBBAFDFDFB3
:108AE000B9D8B1F1A3978E60DFB084F2C8F8F9D994
:108AF000DED89385F14AB183A308B5839A0810B7ED
:108B00009F10D8F1B0BAAEB08AC2B2B68E9EF1FB59
:108B1000D9F41DD8F9D90CF1D8F8F8AD61D9AEFB6C
:108B2000D8F40CF1D8F8F8AD19D9AEFBDFD8F416AB
:108B3000F1D8F8AD8D61D9F4F4ACF59C9C8DDF2BA8
:108B4000BAB6AEFAF8F40BD8F1AED0F8AD51DAAE51
:108B5000FAF8F1D8B9B1B6A3839C08B9B1839AB534
:108B6000AAC0FD3083B79F10B58B93F20202D1AB40
:108B7000DADED8F1B080BAABC0C3B284C1C3D8B119
:108B8000B9F38BA391B609B4D9ABDEB0879CB9A376
:108B9000DDF1B38B8B8B8B8BB087A3A3A3A3B28B9D
:108BA000B69BF2A3A3A3A3A3A3A3A3A3A3F1B087FC
:108BB000B59AA3F39BA3A3DCBAACDFB9A3A3A3A389
:108BC000A3A3A3A3A3A3A3A3A3A3A3A3D8D8D8BBBE
:108BD000B3B7F1AAF9DAFFD9809AAA28B48098A786
:108BE00020B79787A86688F07951F1902C870CA759
:108BF00081976293F071716085940129517990A5F4
:108C0000F1284C6C870C95188578A38390284C6CC0
:108C1000886CD8F3A28200F210A8921980A2F2D92F
:108C200026D8F188A84DD948D896A83980D93CD8FB
:108C30009580A839A68698D92CDA87A72CD8A88938
:108C40009519A980D938D8A88939A980DA3CD8A83B
:108C50002EA83990D90CD8A8953198D90CD8A80944
:108C6000D9FFD801DAFFD89539A9DA26FFD890A81C
:108C70000D8999A810809821DA2ED88999A8318079
:108C8000DA2ED8A886963180DA2ED8A8873180DAF5
:108C90002ED8A88292F34180F1D92ED8A882F31958
:108CA00080F1D92ED882ACF3C0A28022F1A62EA7E3
:108CB0002EA92298A829DAACDEFFD8A2F22AF1A9BF
:108CC0002E8292A8F23180A696F1D900AC8C9C0C31
:108CD00030ACDED0DEFFD88C9CACD010ACDE809205
:108CE000A2F24C82A8F1CAF235F19688A6D900D832
:108CF000F1FF0000000000004FBB610567ACDD3FE5
:108D0000182D4454FB21E93F9BF681D20B73EF3FB2
:108D1000182D4454FB21F93FE2652F227F2B7A3C2A
:108D2000075C143326A6813CBDCBF07A8807703CE3
:108D3000075C143326A6913CC4EB98999999C9BF56
:108D4000711623FEC671BCBF6D9A74AFF2B0B3BF8B
:108D50009AFDDE522DDEADBF2F6C6A2C44B4A2BF4B
:108D60000D5555555555D53FFF8300922449C23FB7
:108D70006E204CC5CD45B73F513DD0A0660DB13FEB
:108D8000EB0D76244B7BA93F11DA22E33AAD903FFD
:108D9000000000000000000050726F6475637420D2
:108DA00049442072656164206173203020696E64DB
:108DB00069636174657320646576696365206973AE
:108DC0002065697468657220696E636F6D70617487
:108DD00069626C65206F7220616E204D5055333092
:108DE00035302E0D0A000000088E0008000000201B
:108DF000180100006C010008208F000818010020F5
:108E0000480700008801000800A24A040000000092
:108E1000000000000102030406070809000000002A
:108E200001020304010203040607080902040608FC
:108E30000000000000000000000000000000000032
:108E40000000000000000000000000000000000022
:108E50000000000000000000000000000000000012
:108E600046000000000000000000000000000000BC
:108E700000000000000000000000000000000000F2
:108E800000000000000000000100000000000000E1
:108E900000000000000000000000000000000000D2
:108EA00000000000000000000000000000000000C2
:108EB00000000000000000000000000000000000B2
:108EC00000000000000000000000000000000000A2
:108ED000000000000000803F0000000000000000D3
:108EE00000000000FF000000FF0000000100000083
:108EF00000000000B8800008AC80000800000000FE
:108F00000000000000000000000000000000000061
:108F1000000000000000000000000000D4800008F5
:0400000508000131BD
:00000001FF
